:020000040800F2
:10000000A878002035020008693A0008C32D0008CE
:10001000653A0008010400081F40000800000000C5
:10002000000000000000000000000000C93E0008C1
:1000300005040008000000006D3A0008CB3E0008EF
:100040004F0200084F0200084F0200084F0200084C
:100050004F0200084F0200084F0200084F0200083C
:100060004F0200084F0200084F0200084F0200082C
:100070004F0200084F0200084F0200084F0200081C
:100080004F0200084F0200084F0200084F0200080C
:100090004F0200084F0200084F0200084F020008FC
:1000A0004F0200084F0200084F0200084F020008EC
:1000B0004F0200084F020008000000004F02000835
:1000C0004F0200084F0200084F0200084F020008CC
:1000D0004F0200084F0200084F0200084F020008BC
:1000E0004F0200084F02000800000000000000005E
:1000F0000000000000000000000000000000000000
:10010000000000004F020008000000004F0200083D
:100110004F02000800000000593F000800000000E6
:100120004F0200084F0200084F0200084F0200086B
:100130004F0200084F0200084F02000800000000B4
:100140004F0200084F0200084F0200084F0200084B
:100150004F0200084F0200084F0200084F0200083B
:100160004F0200084F0200084F0200080000000084
:10017000000000004F020008000000000000000026
:100180004F0200084F0200084F0200084F0200080B
:100190004F02000800F002F800F03CF80AA090E8D6
:1001A000000C82448344AAF10107DA4501D100F032
:1001B00031F8AFF2090EBAE80F0013F0010F18BFC3
:1001C000FB1A43F001031847EC8D00000C8E000071
:1001D000103A24BF78C878C1FAD8520724BF30C873
:1001E00030C144BF04680C60704700000023002445
:1001F00000250026103A28BF78C1FBD8520728BF37
:1002000030C148BF0B6070471FB505F017FA1FBD1E
:1002100010B510BD00F058F81146FFF7F5FF04F0D7
:10022000D9FC00F076F803B4FFF7F2FF03BC00F04E
:100230007BF800000948804709480047FEE7FEE7D1
:10024000FEE7FEE7FEE7FEE7FEE7FEE7FEE7FEE786
:1002500004480549054A064B70470000453F000821
:1002600095010008A8720020A8780020A87400203A
:10027000A87400204FF0000200B51346944696463D
:10028000203922BFA0E80C50A0E80C50B1F12001A9
:10029000BFF4F7AF090728BFA0E80C5048BF0CC057
:1002A0005DF804EB890028BF40F8042B08BF7047B5
:1002B00048BF20F8022B11F0804F18BF00F8012B27
:1002C0007047704770477047754600F029F8AE4692
:1002D00005006946534620F00700854618B020B552
:1002E000FFF7B6FFBDE820404FF000064FF00007D3
:1002F0004FF000084FF0000B21F00701AC46ACE8CE
:10030000C009ACE8C009ACE8C009ACE8C0098D463A
:1003100070470446AFF300802046FFF784FF0000DB
:10032000004870474872002001491820ABBEFEE724
:10033000260002007047000038B5044600200090F7
:10034000206803F0BFF900284FD120688068284951
:10035000084048B1A06D40F01000A065E06D40F08D
:100360000100E065012038BD206803F095F900BF69
:100370002048806800F0E07000F4000080B11E4862
:1003800000681E49B0FBF1F0401C00EB400080000B
:10039000009002E00098401E009000980028F9D1DB
:1003A00000F042FD05461AE0206803F08BF910B911
:1003B000206803F071F900F037FD401B02280ED9C8
:1003C0002068006800F0010048B9A06D40F01000FE
:1003D000A065E06D40F00100E0650120C3E7206802
:1003E000006800F001000028DED00020BBE700001C
:1003F0003F000080000304500C000020400D03006B
:1004000000BFFEE7704772B6704700002DE9FC5F41
:1004100005460C46002001900090FE49E0688842A5
:1004200000D000E000BF00BF95F85400012802D1C1
:100430000220BDE8FC9F012085F8540000BF286819
:1004400003F04AF900287DD167686068052815D84F
:100450006068022806D0032806D0042806D00528A4
:1004600009D105E00C2708E0122706E0182704E070
:100470004FF4807701E0062700BF00BF286821689D
:1004800000F13003C7F3012C03EB8C02136807F073
:100490001F0B4FF01F0C0CFA0BFC23EA0C0307F0A8
:1004A0001F0CC1F3846B0BFA0CFB43EA0B031360C4
:1004B00000BF286803F010F98246286803F0FDF8B1
:1004C0008146BAF1000F3FD1B9F1000FFBD1A0680E
:1004D000B0F1004F0AD121680022286803F00AF920
:1004E0004FF00041286803F02AF908E0A26821686B
:1004F000286803F0FFF80021286803F020F96069FC
:100500002968C968C1F3C101490000FA01F82069EE
:1005100004281AD028682268216900F1600C0CEBCD
:100520008103D3F800C0DFF8F0B20CEA0B0C02F044
:10053000F84B4BF0004B4BEA080B4CEA0B0CC3F8A2
:1005400000C000E0B7E100BFA7E00021286803F089
:10055000ABF8C0F3120030B90021286803F0A4F80A
:10056000C0F3846007E00021286803F09DF890FA4A
:10057000A0F0B0FA80F02168C1F3120119B9216826
:10058000C1F3846104E0216891FAA1F1B1FA81F12B
:10059000884204D100221146286803F0C5F80121E1
:1005A000286803F081F8C0F3120030B901212868EF
:1005B00003F07AF8C0F3846007E00121286803F0B3
:1005C00073F890FAA0F0B0FA80F02168C1F312013C
:1005D00019B92168C1F3846104E0216891FAA1F19D
:1005E000B1FA81F1884204D100220121286803F088
:1005F0009BF80221286803F057F8C0F3120030B9C5
:100600000221286803F050F8C0F3846007E002215B
:10061000286803F049F890FAA0F0B0FA80F0216859
:10062000C1F3120119B92168C1F3846104E02168A2
:1006300091FAA1F1B1FA81F1884204D1002202219C
:10064000286803F071F80321286803F02DF8C0F33F
:10065000120030B90321286803F026F8C0F3846043
:1006600007E00321286803F01FF890FAA0F0B0FA21
:1006700080F02168C1F3120119B92168C1F38461C6
:1006800004E0216891FAA1F1B1FA81F1884204D124
:1006900000220321286803F047F8286803F012F8C5
:1006A000002872D12868E2682168D0F8B030C1F320
:1006B000120C23EA0C0302F0180BDFF860C12CFACD
:1006C0000BFC0CEA010C43EA0C03C0F8B03000BF8D
:1006D0005049E068884258D12368C3F312031BB91C
:1006E0002368C3F3846304E0236893FAA3F3B3FAA3
:1006F00083F35B1C03F01F03092B3ED82368C3F36D
:1007000012031BB92368C3F3846304E0236893FADC
:10071000A3F3B3FA83F35B1C03F01F034FF0010C48
:100720000CFA03FC2368C3F312031BB92368C3F359
:10073000846304E0236893FAA3F3B3FA83F35B1CA6
:1007400003F01F034CEA836C2368C3F312031BB945
:100750002368C3F3846304E0236893FAA3F3B3FA32
:1007600083F35B1C03F01F0303EB43034FF0000B09
:100770004BEA03534CEA03033FE02368C3F312033D
:1007800023B92368C3F3846305E03BE0236893FA4D
:10079000A3F3B3FA83F35B1C03F01F034FF0010CC8
:1007A0000CFA03FC2368C3F312031BB92368C3F3D9
:1007B000846304E0236893FAA3F3B3FA83F35B1C26
:1007C00003F01F034CEA836C2368C3F312031BB9C5
:1007D0002368C3F3846304E0236893FAA3F3B3FAB2
:1007E00083F35B1C03F01F030A3B03EB43034FF04F
:1007F000007B4BEA03534CEA03031946A2682868BE
:1008000002F078FF06492068084088B300BF054819
:10081000806809E000007F4000F0FF03FFFF070051
:10082000000008800003045000F0E07600BF284973
:10083000206888421DD106F40000D0B925492868F7
:10084000884237D146F40001234802F067FF23486D
:1008500000682349B0FBF1F0401C00EB4000800031
:10086000009002E00098401E009000980028F9D106
:1008700020E01C49206888420CD106F0807048B9FD
:1008800014492868884215D146F08071124802F058
:1008900045FF0FE01449206888420BD106F4800020
:1008A00040B90C492868884204D146F480010A48BE
:1008B00002F034FF05E0A86D40F02000A86501209B
:1008C000019000BF002085F8540000BF0198B0E5FA
:1008D000000052C700000450000304500C00002028
:1008E000400D0300000084CB010000800146086831
:1008F000006C70472DE9F84304464FF000080020D3
:10090000009014B90120BDE8F883206920B12020AF
:10091000005D012800D100BFA06D30B9204600F075
:10092000E3F80020E06584F8540020688168C1F392
:10093000407131B120688168644A1140816000BF14
:1009400000BF206802F0C3FEB0B920688168604A29
:10095000114041F08051816000BF5E4800685E49EF
:10096000B0FBF1F0401C4000009002E00098401EF7
:10097000009000980028F9D1206802F0A8FE48B93C
:10098000A06D40F01000A065E06D40F00100E06552
:100990004FF00108206802F09FFE0646A06D00F0AF
:1009A000100000287BD1002EFCD1A06D20F48070B7
:1009B00040F00200A065206802F084FE68B9474854
:1009C00002F080FE48B960684549896821F47C11CD
:1009D0000143434A916000BF00BF607E616B41EA02
:1009E0004030E1680843A16808432021095D40EADE
:1009F00001452020005D012803D1A08C401E45EA5E
:100A00004045A06A28B1208D00F47070E16A084367
:100A100005432068C0683349084028432168C860FE
:100A2000206802F04AFE07462EBB27BB207EE16C01
:100A300041EA803194F8300041EA40052068C068FE
:100A400044F20601884328432168C86094F83800BE
:100A5000012811D1E06B40F00101206C0843616C6A
:100A60000843A16C08432168096940F2FC72914374
:100A700008432168086105E02068006920F0010052
:100A800021680861206901280AD12068006B20F0E4
:100A90000F00E169491E08432168086306E00CE085
:100AA0002068006B20F00F0021680863A06D20F023
:100AB000020040F00100A06505E0A06D40F01000CC
:100AC000A0654FF0010840461DE70000C0FFFF5F32
:100AD000C0FFFF7F0C000020400D03000000045009
:100AE0000003045007C0F0FF10B5A0B00446142165
:100AF0001BA8FFF7BFFB682101A8FFF7BBFB22493A
:100B0000206888423DD14FF48040019080031890C6
:100B100003200290012103910821049107210591EE
:100B2000022106910791C905089101A800F0C0FBB8
:100B300008B1FFF768FC00BF1448C06C40F40050D7
:100B40001249C8640846C06C00F40050009000BF11
:100B500000BF00BF0846C06C40F00100C8640846F2
:100B6000C06C00F00100009000BF00BF20201B906F
:100B70000B201C9000201D901BA94FF0904000F00E
:100B800065F820B010BD00000000045000100240C5
:100B900070B50446206802F09FFD00283FD100BFD9
:100BA00094F85400012801D1022070BD012084F87E
:100BB000540000BF2046FFF7BFFB054655BBA06DA4
:100BC00040F60161884340F48070A065A06D00F498
:100BD0008050B0F5805F04D1E06D20F00600E06544
:100BE00001E00020E0651C202168086000BF0020B3
:100BF00084F8540000BF2068C06800F0007028B17D
:100C0000A06D20F4005040F48050A065206802F0F0
:100C100069FD05E000BF002084F8540000E00225D3
:100C20002846C2E770B5044600F0FEF806462546A1
:100C3000681C10B104480078054400BF00F0F4F8C7
:100C4000801BA842FAD370BD0800002078B5034687
:100C50000A460021C5E001268E40156805EA060413
:100C6000002C73D0157905F00305012D04D01579FA
:100C700005F00305022D13D198684E000325B540F9
:100C8000A8434E00D568B5402843986058680125B0
:100C90008D40A8431579C5F300158D402843586051
:100CA000157905F00305032D09D0D8684E000325FA
:100CB000B540A8434E009568B5402843D8601579E3
:100CC00005F00305022D13D1CE0803F1200555F8D8
:100CD00026004D07EE0E0F25B540A8434E07F60E31
:100CE0001569B5402843CE0803F1200545F82600D4
:100CF00018684E000325B540A843157905F0030593
:100D00004E00B54028431860556805F44035002D65
:100D100066D000BF364D2D6E45F00105344E356668
:100D200035462D6E05F00105009500BF00BF4FEA66
:100D3000B6358E0855F826008D072E0F0F25B540C5
:100D4000A843B3F1904F02D1002515E048E0294DAA
:100D5000AB4201D101250FE0274DAB4201D1022565
:100D60000AE0264DAB4201D1032505E0244DAB42FC
:100D700001D1042500E007258E07360FB540284332
:100D8000204D8E0845F826001F4D2868A043556861
:100D900005F4801505B120431B4D28602D1D2868E2
:100DA000A043556805F4001505B12043164D2D1DCF
:100DB0002860154D2D1F2868A043556805F400359F
:100DC00005B12043104D2D1F28602D1F2868A0431A
:100DD000556805F4803505B120430B4D083D28606A
:100DE000491C1568CD40002D7FF435AF78BD00005B
:100DF000001002400004004800080048000C0048B1
:100E00000010004808000140080401400246136930
:100E10000B400BB1012000E0002070470AB1816156
:100E200000E08162704700000148006870470000E0
:100E300000000020024692F8410020282DD100BF7A
:100E400092F84000012801D102207047012082F869
:100E5000400000BF242082F841001068006820F0A4
:100E60000100136818601068006820F4805013684F
:100E700018601068006808431368186010680068FC
:100E800040F0010013681860202082F8410000BF84
:100E9000002082F8400000BFD7E70220D5E710B558
:100EA00002460B4692F8410020282AD100BF92F852
:100EB0004000012801D1022010BD012082F840002D
:100EC00000BF242082F841001068006820F0010073
:100ED000146820601068016821F4706141EA032100
:100EE000106801601068006840F00100146820601C
:100EF000202082F8410000BF002082F8400000BF9F
:100F0000DAE70220D8E7000010B504460CB901204A
:100F100010BD94F8410028B9002084F84000204614
:100F200000F05EF8242084F841002068006820F07A
:100F3000010021680860606820F070602168086125
:100F40002068806820F4004021688860E0680128FB
:100F500005D1A06840F400402168886004E0A068E2
:100F600040F4044021688860E068022806D12068C7
:100F7000406840F400602168486005E020684068EF
:100F800020F40060216848602068406813490843E5
:100F9000216848602068C06820F400402168C8606B
:100FA000D4E904010843A16940EA01202168C8602E
:100FB000D4E907010843216808602068006840F010
:100FC00001002168086000206064202084F841004E
:100FD0000020206384F8420000BF99E700800002EF
:100FE00010B5A0B0044614211BA8FFF743F96821EF
:100FF00001A8FFF73FF91D492068884234D14FF41A
:10100000801001900020119001A800F051F908B162
:10101000FFF7F9F900BF1648C06C40F00200144910
:10102000C8640846C06C00F00200009000BF00BF1A
:101030004FF440601B9012201C9000201D90032054
:101040001E901F901BA90B48FFF700FE00BF084829
:10105000C06D40F002000649C8650846C06D00F04A
:101060000200009000BF00BF20B010BD008400400F
:101070000010024000040048034800680349097852
:101080000844014908607047000000200800002063
:1010900010B50024032000F0A9F80F2000F008F894
:1010A00008B1012401E000F02FF8204610BD000037
:1010B00070B50446002511480078D8B10F48007873
:1010C0004FF47A71B1FBF0F00D490968B1FBF0F60D
:1010D000304601F03DFB58B9102C07D200222146C2
:1010E000501E00F045F80748046004E0012502E0C6
:1010F000012500E00125284670BD00000800002001
:101100000C0000200400002008B500BF0D48006E50
:1011100040F001000B4908660846006E00F001002F
:10112000009000BF00BF00BF0846806D40F08050B7
:1011300088650846806D00F08050009000BF00BFB9
:1011400008BD0000001002400146084600280DDBE3
:1011500000BF00BF00F01F0301229A4043099B001B
:1011600003F1E023C3F8002100BF00BF00BF7047B8
:101170002DE9F05F80460D461646002702F052FF2B
:10118000074639462A46334601F00700C0F1070AF0
:10119000BAF1040F02D94FF0040A01E0C0F1070AC6
:1011A000D14600F1040ABAF1070F02D24FF0000A4B
:1011B00001E0A0F1030AD4464FF0010A0AFA09FA45
:1011C000AAF1010A0AEA020A0AFA0CFA4FF0010B24
:1011D0000BFA0CFBABF1010B0BEA030B4AEA0B0415
:1011E0002146404602F026FFBDE8F09F00BF00F018
:1011F0000702064B19684FF6FF031940044B0B43D7
:1012000043EA0221014B196000BF70470CED00E07A
:101210000000FA050246B2F5007F2AD11D48006899
:1012200000F4C060B0F5007F32D01A48006820F4A6
:10123000C06040F40070174B1860174800683223F4
:101240005843164BB0FBF3F0411C00E0491E114817
:10125000406900F48060B0F5806F01D10029F5D1BC
:101260000C48406900F48060B0F5806F10D1032015
:1012700070470848006800F4C060B0F5806F07D080
:101280000448006820F4C06040F48060014B18609E
:101290000020EDE7007000400C00002040420F00ED
:1012A0000248006800F4C060704700000070004011
:1012B0002DE9F84304460025A846208800F4006084
:1012C000B0F5006F26D1E06C68B1B0F5000F03D027
:1012D000B0F5400F0ED10CE0F748C06840F4803004
:1012E000F549C86008E00021201D02F0C1FB054659
:1012F00002E001E0012500BF00BF55B9EE4888308B
:10130000006820F44000E16C0843EB49C1F8880014
:1013100000E0A846206800F40030B0F5003F75D129
:101320004FF00009E448806D012121EA107078B186
:1013300000BFE148806D40F08050DF498865084675
:10134000806D00F08050009000BF00BF4FF0010999
:10135000DA48006840F48070D8490860FFF764FDFF
:10136000074606E0FFF760FDC01B022801D90325F0
:1013700005E0D248006800F480700028F2D000BF79
:101380007DBBCD489030006800F44076CEB1606EF1
:10139000B04216D0C8489030006820F44076C64865
:1013A000D0F8900040F48030C349C1F8900008465E
:1013B000D0F8900020F48030C1F890000846C0F8C2
:1013C000906006F00100A8B1FFF72EFD074609E086
:1013D000FFF72AFDC01B41F28831884202D903255C
:1013E00007E016E0B4489030006800F002000028E2
:1013F000EED000BF5DB9B0489030006820F4407076
:10140000616E0843AC49C1F8900003E00CE0A846C7
:1014100000E0A846B9F1010F05D1A748806D20F082
:101420008050A549886500BF207800F0010048B1D0
:10143000A1488830006820F00300216A08439E49D3
:10144000C1F88800207800F00200022809D19A48EB
:101450008830006820F00C00616A08439649C1F8A2
:101460008800207800F00400042809D192488830D0
:10147000006820F03000A16A08438F49C1F8880055
:10148000207800F00800082809D18B4888300068CF
:1014900020F0C000E16A08438749C1F8880020783D
:1014A00000F02000202809D183488830006820F40B
:1014B0004060216B08438049C1F88800208800F40F
:1014C0000070B0F5007F09D17B488830006820F4B7
:1014D0004020616C08437849C1F88800208800F4F6
:1014E0008060B0F5806F09D173488830006820F4BF
:1014F0004010A16C08437049C1F88800207800F0C2
:101500004000402809D16C488830006820F44050E1
:10151000616B08436849C1F88800207800F08000BA
:10152000802809D164488830006820F44040A16BCD
:1015300008436149C1F88800208800F48070B0F544
:10154000807F09D15C488830006820F44030E16B2E
:1015500008435949C1F88800206800F48010B0F5AC
:10156000801F09D154489C30006820F00300216C92
:1015700008435149C1F89C00208800F40050B0F5A0
:10158000005F1FD14C488830006820F04060216D1A
:101590000843494988310860206DB0F1006F06D1D9
:1015A0004548C06840F480104349C8600AE0206D97
:1015B000B0F1806F06D10121201D02F059FA0546D5
:1015C00005B1A846206800F40020B0F5002F1FD117
:1015D00039488830006820F04060616D0843364922
:1015E00088310860606DB0F1006F06D13248C06884
:1015F00040F480103049C8600AE0606DB0F1806F3F
:1016000006D10121201D02F033FA054605B1A84696
:10161000206800F48020B0F5802F1FD12648883044
:10162000006820F04060A16D0843234988310860BC
:10163000A06DB0F1006F06D11F48C06840F4801063
:101640001D49C8600AE0A06DB0F1806F06D101218C
:10165000201D02F00DFA054605B1A846208800F4C9
:101660008040B0F5804F14D113488830006820F0D6
:101670004050E16D0843104988310860E06DB0F1D9
:10168000805F06D10221201D02F0F2F9054605B166
:10169000A846206800F48030B0F5803F09D10648A4
:1016A0008830006820F00040216E08430249C1F8EC
:1016B00088004046BDE8F8830010024000700040FA
:1016C0002DE9F04104460D4614B90120BDE8F08132
:1016D0006348006800F00700A8420ED26048006826
:1016E00020F0070028435E4908600846006800F0C3
:1016F0000700A84201D00120E8E7207800F00200AE
:1017000002280ED15749A068896801F0F00188428B
:1017100007D95448806820F0F000A1680843514977
:101720008860207800F0010078B36068032806D153
:101730004C48006800F00070D8B90120C6E7606826
:10174000022806D14748006800F4003088B901201B
:10175000BCE7606830B94348006800F0020040B957
:101760000120B3E73F48006800F4806008B9012019
:10177000ACE73C48806820F00300616808433949C1
:101780008860FFF751FB064609E010E0FFF74CFBCD
:10179000801B41F28831884201D9032096E7314805
:1017A000806800F00C006168B0EB810FEED120780A
:1017B00000F0020002280ED12A49A068896801F0D1
:1017C000F001884207D22748806820F0F000A16825
:1017D0000843244988602248006800F00700A842B6
:1017E0000ED91F48006820F0070028431C490860F4
:1017F0000846006800F00700A84201D0012065E714
:10180000207800F00400042807D11648806820F4EE
:10181000E060E168084313498860207800F0080020
:10182000082808D10F48806820F46050216940EAF8
:10183000C1000C49886000F01DF80A498968C1F3AD
:101840000311094A515C01F01F01C84007490860B3
:1018500007480068FFF72CFC0746384636E70000CB
:101860000020024000100240505600080C000020EA
:1018700004000020F0B500230020DFF8D4C0DCF81D
:1018800008C00CF00C01DFF8C8C0DCF80CC00CF08C
:10189000030719B10C291ED1012F1CD1DFF8B0C0EC
:1018A000DCF800C00CF0080CBCF1000F06D1DFF82A
:1018B000A0C0DCF894C0CCF3032305E0DFF890C0AF
:1018C000DCF800C0CCF30313DFF888C05CF82330E9
:1018D00041B9184606E0042901D11F4802E0082951
:1018E00000D11E480C2932D1DFF864C0DCF80CC0EE
:1018F0000CF00304012C09D0022C02D0032C04D1DB
:1019000001E0154A04E0154A02E000BF1A4600BF94
:1019100000BFDFF83CC0DCF80CC0CCF3021C0CF1BB
:101920000106DFF82CC0DCF80CC0CCF3062C0CFB55
:1019300002FCBCFBF6F2DFF818C0DCF80CC0CCF3FC
:10194000416C0CF1010C4FEA4C05B2FBF5F0F0BD17
:1019500000100240685600080024F40000127A00CB
:101960002DE9F843044614B90120BDE8F883F9488D
:10197000806800F00C06F748C06800F00307207884
:1019800000F01000102877D11EB10C2E76D1012F57
:1019900074D1F048006800F0020018B1A06908B9DD
:1019A0000120E2E7EB48216A006800F0080020B15E
:1019B000E848006800F0F00005E0E6489430006870
:1019C00000F47060000981421FD9206A02F014F906
:1019D00008B10120C9E700BFDE48006840F00800F8
:1019E000DC4908600846006820F0F000216A0843DE
:1019F000D849086000BF0846406820F47F40E1698C
:101A000040EA0120D34948601FE000BFD148006888
:101A100040F00800CF4908600846006820F0F00058
:101A2000216A0843CB49086000BF0846406820F49B
:101A30007F40E16940EA0120C64948602EB9206A2A
:101A400002F0DAF808B101208FE7FFF713FFC14970
:101A50008968C1F30311C04A515C01F01F01C840FD
:101A6000BE490860BE480068FFF722FB8046B8F117
:101A7000000F4ED0404678E74BE0FFE7A06980B307
:101A8000B448006840F00100B2490860FFF7CCF9A3
:101A9000054606E0FFF7C8F9401B022801D90320DC
:101AA00063E7AC48006800F002000028F2D000BFF5
:101AB000A848006840F00800A64908600846006889
:101AC00020F0F000216A0843A249086000BF0846E0
:101AD000406820F47F40E16940EA01209D49486068
:101AE00017E0FFE79B48006820F001009949086073
:101AF000FFF79AF9054606E0FFF796F9401B022822
:101B000001D9032031E79348006800F00200002863
:101B1000F2D1207800F0010000285CD0082E03D01C
:101B20000C2E0AD1032F08D18A48006800F4003037
:101B300088B3606878BB012017E700BF6068B0F524
:101B4000803F06D18348006840F4803081490860B6
:101B50001AE06068B0F5A02F0BD17E48006840F411
:101B600080207C4908600846006840F480300860A6
:101B70000AE07848006820F480307649086008461A
:101B8000006820F48020086000BF606890B1FFF713
:101B90004BF9054607E01EE0FFF746F9401B6428B5
:101BA00001D90320E1E66B48006800F4003000280A
:101BB000F2D010E0FFF738F9054606E0FFF734F9F8
:101BC000401B642801D90320CFE66248006800F476
:101BD00000300028F2D1207800F00200022852D113
:101BE000042E03D00C2E14D1022F12D159480068B4
:101BF00000F4806018B1E06808B90120B5E65548E6
:101C0000406820F0FE40217C40EA01605149486074
:101C100039E0E06800B34F48006840F480704D49F7
:101C20000860FFF701F9054606E0FFF7FDF8401BE5
:101C3000022801D9032098E64648006800F4806035
:101C40000028F2D04348406820F0FE40217C40EA62
:101C500001604049486016E03E48006820F480700A
:101C60003C490860FFF7E0F8054606E0FFF7DCF8BE
:101C7000401B022801D9032077E63648006800F4AB
:101C800080600028F2D1207800F00800082836D1C2
:101C90006069D0B12F489430006840F001002D49B0
:101CA000C1F89400FFF7C0F8054606E0FFF7BCF85E
:101CB000401B022801D9032057E6264894300068CB
:101CC00000F002000028F1D019E0224894300068AA
:101CD00020F001001F49C1F89400FFF7A5F8054660
:101CE00006E0FFF7A1F8401B022801D903203CE6DB
:101CF00018489430006800F002000028F1D12078E4
:101D000000F00400042872D14FF000091148806DE2
:101D100000F0805078B900BF0E48806D40F08050D0
:101D20000C4988650846806D00F08050009000BF27
:101D300000BF4FF001090B48006800F4807000BB41
:101D40000848006840F4807006490860FFF76CF8A6
:101D5000054610E000100240505600080C0000201C
:101D60000400002000700040FFF75EF8401B0228CE
:101D700001D90320F9E5CA48006800F48070002802
:101D8000F2D000BFA068012808D1C648006840F022
:101D90000100C4499039C1F8900021E0A0680528ED
:101DA0000FD1C048006840F00400BE499039C1F826
:101DB00090000846D0F8900040F00100C1F8900073
:101DC0000EE0B848006820F00100B6499039C1F82B
:101DD00090000846D0F8900020F00400C1F8900070
:101DE00000BFA068A0B1FFF71FF8054609E02EE08C
:101DF000FFF71AF8401B41F28831884201D90320CD
:101E0000B3E5A848006800F002000028F0D012E016
:101E1000FFF70AF8054608E0FFF706F8401B41F215
:101E20008831884201D903209FE59E48006800F070
:101E300002000028F0D1B9F1010F07D1994890387C
:101E4000806D20F0805097499039886500BF2078D8
:101E500000F02000202838D1606AD8B191480830BD
:101E6000006840F001008F499039C1F89800FEF7F2
:101E7000DBFF054606E0FEF7D7FF401B022801D92D
:101E8000032072E587480830006800F0020000284F
:101E9000F1D01AE083480830006820F00100814941
:101EA0009039C1F89800FEF7BFFF054606E0FEF73F
:101EB000BBFF401B022801D9032056E579480830B2
:101EC000006800F002000028F1D1A06A00287DD04F
:101ED000A06A02287BD173489038C76807F00301D5
:101EE000E06A814225D107F07001206B401EB1EB02
:101EF000001F1ED107F4FE41606BB1EB002F18D11B
:101F000007F078413820005DB1EBC06F11D107F4C4
:101F1000C001A08F0122C2EB5000B1EB405F08D19D
:101F200007F0C0614020005DC2EB5000B1EB406F94
:101F300066D00C2E62D05B489038006800F080605C
:101F400008B1012011E557489038006820F08070F2
:101F5000544990390860FEF767FF054606E0FEF732
:101F600063FF401B022801D90320FEE44D4890384E
:101F7000006800F000700028F1D1D4E90B10401E79
:101F800041EA0011606B41EA0021A08F0122C2EBFF
:101F9000500041EA40514020005DC2EB500041EA50
:101FA00040613820005D41EAC0603E499039C9680F
:101FB0003D4A114008433B499039C86008460068D3
:101FC00040F0807008600846C06801E053E03DE0E2
:101FD00040F08070C860FEF727FF054606E0FEF778
:101FE00023FF401B022801D90320BEE42D4890386E
:101FF000006800F000700028F1D04FE00120B4E448
:1020000028489038006800F00070A0BB2548903840
:10201000006840F080702349903908600846C06825
:1020200040F08070C860FEF7FFFE054606E0FEF750
:10203000FBFE401B022801D9032096E41948903882
:10204000006800F000700028F1D027E00C2E23D0AB
:1020500014489038006820F0807012499039086068
:10206000FEF7E2FE054607E0FEF7DEFE401B022813
:1020700002D9032079E411E00A489038006800F0A2
:1020800000700028F0D107489038C0680749084020
:1020900004499039C86001E0012066E4002064E44E
:1020A00000700040901002408C809D01FCFFEEFE0D
:1020B00070B504460CB9012070BD606A38B960681B
:1020C000B0F5827F00D105E00021E16102E000214E
:1020D000216161610021A16294F85D0028B90020AE
:1020E00084F85C00204600F05BF8022084F85D0074
:1020F0002068006820F0400021680860E068B0F5C2
:10210000E06F01D9002501E04FF48055E068B0F59B
:10211000706F05D0E068B0F5E06F01D00021A162DA
:10212000A08800F48270218901F404410843217CD5
:1021300001F002010843217D01F001010843218BD8
:1021400001F400710843217F01F038010843202188
:10215000095D01F080010843218D01F4005108431D
:10216000216808600421A06901EA104094F8241055
:1021700001F01001084394F8341001F008010843FD
:10218000A18901F47061084305F480510843216876
:10219000486000202066012084F85D0000208BE765
:1021A00010B586B00446142101A8FEF763F82F4944
:1021B000206888422AD100BF2D48006E40F480502C
:1021C0002B4908660846006E00F48050009000BF5E
:1021D00000BF00BF0846C06C40F00100C86408465C
:1021E000C06C00F00100009000BF00BFC220019051
:1021F0000220029000200390032004900520059007
:1022000001A94FF09040FEF721FD2DE0194920680B
:10221000884229D100BF1648806D40F4804014499F
:1022200088650846806D00F48040009000BF00BFC4
:1022300000BF0846C06C40F00200C8640846C06C8D
:1022400000F00200009000BF00BF4FF4604001901A
:1022500002200290002003900320049005200590A6
:1022600001A90548FEF7F2FC06B010BD00300140A0
:102270000010024000380040000400482DE9F843F7
:1022800004460F4616461D46FEF7CEFD8046B14673
:1022900094F85D00012802D00220BDE8F88307B160
:1022A0000EB90120F9E700BF94F85C00012801D1C4
:1022B0000220F2E7012084F85C0000BF032084F8CC
:1022C0005D0000202066A763A687E6872064A4F847
:1022D0004400A4F846002065E064A068B0F5004F13
:1022E0000BD12068006820F0400021680860206859
:1022F000006840F48040216808602068006800F0B1
:102300004000402805D02068006840F04000216867
:102310000860E068B0F5E06F37D9606810B1B9F1D6
:10232000010F09D1A06B00882168C860A06B801CD8
:10233000A063E08F401EE08723E02068806800F003
:10234000020002280AD1A06B00882168C860A06B37
:10235000801CA063E08F401EE08712E0FEF764FD62
:10236000A0EB0800A84201D3681C00B94DB90120B8
:1023700084F85D0000BF002084F85C0000BF0320EB
:102380008BE7E08F0028D8D152E0606810B1B9F136
:10239000010F17D1E08F01280AD9A06B00882168AE
:1023A000C860A06B801CA063E08F801EE08709E0FE
:1023B000A06B007821680873A06B401CA063E08FBD
:1023C000401EE08731E02068806800F002000228AB
:1023D00018D1E08F01280AD9A06B00882168C86055
:1023E000A06B801CA063E08F801EE0871DE0A06BC7
:1023F000007821680873A06B401CA063E08F401E2A
:10240000E08712E0FEF710FDA0EB0800A84201D320
:10241000681C00B94DB9012084F85D0000BF0020A0
:1024200084F85C0000BF032037E7E08F0028CAD1A2
:1024300042462946204601F02DFC08B120202066A6
:10244000A06850B900BF002000902068C0680090CC
:1024500020688068009000BF00BF012084F85D0004
:1024600000BF002084F85C0000BF206E08B101208E
:1024700013E7002011E72DE9FE4F04460F46904672
:102480001D460C9E01200090FEF7CEFC824694F87B
:102490005DB060680190A9460295BBF1010F0BD0B9
:1024A0000198B0F5827F04D1A06810B9BBF1040F88
:1024B00002D00220BDE8FE8F1FB1B8F1000F00D09E
:1024C0000DB90120F6E700BF94F85C00012801D1A6
:1024D0000220EFE7012084F85C0000BF94F85D0063
:1024E000042802D0052084F85D0000202066C4F88E
:1024F0004080A4F84650A4F84450A763E587A58718
:10250000E0642065E068B0F5E06F02D80298012829
:1025100006D92068406820F480502168486005E0B2
:102520002068406840F48050216848602068006856
:1025300000F04000402805D02068006840F04000CE
:1025400021680860E068B0F5E06F56D9606810B1A6
:10255000B9F1010F09D1A06B00882168C860A06B98
:10256000801CA063E08F401EE0873EE0206880680A
:1025700000F00200022810D1E08F70B1009801280D
:102580000BD1A06B00882168C860A06B801CA06381
:10259000E08F401EE087002000902068806800F0F7
:1025A000010080B1B4F8460068B12068C068216CB1
:1025B0000880206C801C2064B4F84600401EA4F8FB
:1025C000460001200090FEF72FFCA0EB0A00B0426D
:1025D0000BD3701C48B1012084F85D0000BF0020BF
:1025E00084F85C0000BF032064E7E08F0028BDD1C1
:1025F000B4F846000028B9D18DE0606810B1B9F197
:10260000010F17D1E08F01280AD9A06B008821683B
:10261000C860A06B801CA063E08F801EE08709E08B
:10262000A06B007821680873A06B401CA063E08F4A
:10263000401EE08768E02068806800F00200022801
:102640001ED1E08FE0B10098012819D1E08F012858
:102650000AD9A06B00882168C860A06B801CA063A9
:10266000E08F801EE08709E0A06B00782168087386
:10267000A06B401CA063E08F401EE087002000900C
:102680002068806800F0010058B3B4F8460040B3F9
:10269000B4F84600012816D92068C068216C08806B
:1026A000206C801C2064B4F84600801EA4F846000C
:1026B000B4F84600012812D82068406840F48050E1
:1026C000216848600BE02068007B216C0870206C5A
:1026D000401C2064B4F84600401EA4F846000120C7
:1026E0000090FEF7A1FBA0EB0A00B04201D3701CE2
:1026F00000B94EB9012084F85D0000BF002084F8C5
:102700005C0000BF0320D5E6E08F002893D1B4F829
:10271000460000288FD152463146204601F0BAFAD1
:1027200040B12020206600BF002084F85C0000BF7C
:102730000120BFE6012084F85D0000BF002084F87E
:102740005C0000BF206E08B10120B3E60020B1E6B6
:1027500070B504462546681EB0F1807F01D3012084
:102760000FE0681E4FF0E02148610F214FF0FF306D
:1027700001F060FC00204FF0E02188610720086133
:10278000002070BD704770477047000030B50246AA
:102790000B4600BF92F83C00012801D1022030BD59
:1027A000012082F83C0000BF022082F83D00106842
:1027B000416810688468174D1068A84203D121F45D
:1027C00070015868014321F07001186801431068D6
:1027D0004160104D1068A8420BD01068B0F1804FD6
:1027E00007D00D4D1068A84203D00C4D1068A842C8
:1027F00005D124F0800498680443106884600120A7
:1028000082F83D0000BF002082F83C0000BF00BFFE
:10281000C5E70000002C01400004004000400140DA
:1028200010B504460CB9012010BD94F83D0028B93C
:10283000002084F83C00204600F02AF8022084F8AA
:102840003D00211D206801F08FFB012084F8480025
:1028500000BF84F83E0001213F2001554020015572
:1028600041200155422001554320015500BF00BFC2
:10287000012084F844004520015546200155472099
:10288000015500BF012084F83D000020CCE7000086
:1028900038B504460D492068884215D100BF0C4860
:1028A000806D40F010000A4988650846806D00F090
:1028B0001000009000BF00BF002211463620FEF736
:1028C00057FC3620FEF740FC38BD000000100040E9
:1028D00000100240014691F83D00012801D001207E
:1028E0007047022081F83D000868C06840F0010090
:1028F0000B68D860144B086898420BD00868B0F198
:10290000804F07D0114B0868984203D0104B0868DD
:10291000984210D1086880680E4B00EA0302062A2C
:102920000FD0B2F5803F0CD00868006840F001007D
:102930000B68186005E00868006840F001000B684B
:1029400018600020CCE70000002C0140000400408B
:1029500000400140070001002DE9F04104460D460A
:1029600014B90120BDE8F08194F83D0028B9002099
:1029700084F83C00204600F055F8022084F83D0021
:10298000206880682649084021688860211D2068E9
:1029900001F0EAFA2068D0F808802068866920688B
:1029A000076A286840EA080840F203308643A969AC
:1029B000A86840EA0120064340F60C4086434FF2E7
:1029C000F0008643E969E86840EA01200643286987
:1029D0000001296A40EA0130064327F0220727F068
:1029E00088076969686840EA011007432068C0F8F1
:1029F00008802068866120680762012084F848000A
:102A000084F83E0001213F200155012084F8440054
:102A100045200155012084F83D000020A2E7000078
:102A2000F8BFFEFF10B586B00446142101A8FDF7DB
:102A300021FC1849206888422AD100BF1648006E40
:102A400040F40060144908660846006E00F4006017
:102A5000009000BF00BF00BF0846C06C40F00100FE
:102A6000C8640846C06C00F00100009000BF00BFC1
:102A70004FF4407001900220029001200390022048
:102A800004900120059001A94FF09040FEF7DEF878
:102A900006B010BD002C0140001002402DE9F043AB
:102AA00004460D4694F83E603F20075D94F844804C
:102AB000452010F804906DB9012E02D1B8F1010F34
:102AC00002D00120BDE8F083022084F83E0084F8A3
:102AD000440025E0042D0CD1012F02D1B9F1010FE2
:102AE00001D00120EEE702213F200155452001558C
:102AF00016E0012E07D1012F05D1B8F1010F02D147
:102B0000B9F1010F01D00120DCE7022084F83E007A
:102B100002213F200155022084F844004520015540
:102B200015B1042D0CD105E001220021206801F02F
:102B300065FA10E001220421206801F05FFA0AE042
:102B400001220021206801F059FA012204212068A5
:102B500001F054FA00BF00BF2068006840F0010097
:102B6000216808600020ADE7704770B50446206812
:102B7000C6682068056905F00200022819D106F030
:102B80000200022815D1401F21680861012020772A
:102B90002068806900F0030018B12046FFF7E4FFC9
:102BA00005E0204600F0ADF8204600F0ABF800202C
:102BB000207705F00400042819D106F00400042849
:102BC00015D1C04321680861022020772068806900
:102BD00000F4407018B12046FFF7C6FF05E020461C
:102BE00000F08FF8204600F08DF80020207705F0E7
:102BF0000800082819D106F00800082815D1C0439C
:102C000021680861042020772068C06900F0030073
:102C100018B12046FFF7A8FF05E0204600F071F844
:102C2000204600F06FF80020207705F010001028F3
:102C300019D106F01000102815D1C0432168086191
:102C4000082020772068C06900F4407018B1204641
:102C5000FFF78AFF05E0204600F053F8204600F019
:102C600051F80020207705F0010048B106F001007E
:102C700030B16FF0010021680861204600F044F88F
:102C800005F08000802804D005F40050B0F5005F06
:102C90000AD106F08000802806D16FF40250216826
:102CA00008612046FFF76FFD05F48070B0F5807F66
:102CB0000AD106F08000802806D16FF48070216868
:102CC00008612046FFF75EFD05F04000402809D16D
:102CD00006F04000402805D1C04321680861204625
:102CE00000F06EF805F02000202809D106F0200041
:102CF000202805D1C043216808612046FFF744FD24
:102D000070BD70477047000010B5044622488442E9
:102D100040D122480068406A2149086001F0A8F9C2
:102D200001F000FB1F490968012923D11C490968EA
:102D30001D4A1268881A002801DB014600E0414262
:102D40000E2917DD16480068174908601448016805
:102D500016480268A0F5805040F822101448016817
:102D600012480068134A42F8201010480068401CBE
:102D70000E49086002211048FEF748F810B90220F9
:102D80000E49086001210C48FEF740F810B90320F5
:102D90000A49086010BD000054020020080200200B
:102DA0003C0000202400002040000020A022002041
:102DB00010000020A002002000040048780000203D
:102DC000704700BFFEE72DE9F04107460C46154667
:102DD0001E462A2000F013FC384600F001FC28466D
:102DE00000F0FEFB2B2000F00AFC04F1220188B267
:102DF00000F0F6FB06F1220188B200F0F1FB2C2076
:102E000000F0FDFBBDE8F0812DE9FF4F85B0814664
:102E10008A460020039083460798A0EB090508988E
:102E2000A0EB0A06CDF80890CDF804A0002D01DD36
:102E3000012705E00DB9002702E04FF0FF376D4292
:102E4000002E02DD4FF0010806E016B94FF0000831
:102E500002E04FF0FF387642B54201DD2C4600E03B
:102E60003446002004901EE0019A91B2029A90B27A
:102E7000129A00F01FF8039828440390B344039873
:102E8000A04205DD0398001B03900298384402908D
:102E9000A34504DDABEB040B01984044019004987A
:102EA000401C80B20490611C04988842DCDB09B0AD
:102EB000BDE8F08F70B504460D4616462B462246F7
:102EC00029462046FFF77FFF304600F089FB70BDA2
:102ED0002DE9F84305460E4617469846089C3346AA
:102EE0003A46314628460094FFF78EFF43462A466D
:102EF000314628460094FFF787FF43463A4641464D
:102F000028460094FFF780FF43463A46314638464C
:102F10000094FFF779FFBDE8F8832DE9F0470646F6
:102F20000F4614461D46DDF820A0681E83B2601EC1
:102F300082B239463046FFF746FFB8460EE0B1464A
:102F400006E0504600F04CFB09F101001FFA80F941
:102F5000A145F6DB08F101001FFA80F8A845EEDB79
:102F6000BDE8F08700B587B000BF1048C06C40F0E6
:102F700002000E49C8640846C06C00F002000190CF
:102F800000BF00BF4FF42040029001200390049046
:102F90000220059002A90648FDF758FE0122602193
:102FA0000348FDF73BFF07B000BD000000100240E2
:102FB000000400480EB5FFF7D5FF002208214FF0AE
:102FC0009040FDF72BFF1E2001F076F90122082129
:102FD0004FF09040FDF722FF642001F06DF90022D0
:102FE0004FF48051B648FDF719FF642001F064F9F1
:102FF000112000F004FB362000F001FB702000F0EF
:10300000F8FA3A2000F0FBFA052000F0F2FAB220BC
:1030100000F0F5FA0C2000F0ECFA0C2000F0E9FAD0
:10302000002000F0E6FA332000F0E3FA332000F04D
:10303000E0FAB72000F0E3FA352000F0DAFABB201E
:1030400000F0DDFA352000F0D4FAC02000F0D7FA05
:103050002C2000F0CEFAC22000F0D1FA012000F0BE
:10306000C8FAC32000F0CBFA132000F0C2FAC42043
:1030700000F0C5FA202000F0BCFAC62000F0BFFA2C
:103080000F2000F0B6FAD02000F0B9FAA42000F02A
:10309000B0FAA12000F0ADFAD62000F0B0FAA120DD
:1030A00000F0A7FAE02000F0AAFAF02000F0A1FA60
:1030B000002000F09EFA042000F09BFA042000F0AB
:1030C00098FA042000F095FA052000F092FA2920E1
:1030D00000F08FFA332000F08CFA3E2000F089FADD
:1030E000382000F086FA122000F083FA122000F057
:1030F00080FA282000F07DFA302000F07AFAE120F2
:1031000000F07DFAF02000F074FA072000F071FA68
:103110000A2000F06EFA0D2000F06BFA0B2000F090
:1031200068FA072000F065FA282000F062FA3320E0
:1031300000F05FFA3E2000F05CFA362000F059FA09
:10314000142000F056FA142000F053FA292000F061
:1031500050FA322000F04DFA212000F050FA1120F0
:1031600000F04DFA782001F0A7F8292000F047FA86
:103170004FF6FF70AC234FF4A07200210090084678
:10318000FFF7CBFE00201E2340F2271205210090FE
:10319000D720FFF79DFE002017234FF496720C21D5
:1031A0000090501FFFF794FE4FF4FC601D234FF476
:1031B000937206210090D820FFF7AFFE0020202157
:1031C0004FF6FF724FF47843CDE9002102903DA203
:1031D00001460A2000F0E3F9002020214FF6FF729B
:1031E0004FF47843CDE90021029038A221210A2032
:1031F00000F0D5F9002020214FF6FF724FF47843FC
:10320000CDE90021029034A221214FF4827000F018
:10321000C6F9002020214FF6FF724FF47843CDE924
:10322000002102902DA242210A2000F0B8F90020CE
:1032300020214FF6FF724FF47843CDE90021029030
:1032400025A24221C82000F0AAF9002020214FF633
:10325000FF724FF47843CDE90021029021A263214F
:103260000A2000F09CF9002020214FF6FF724FF455
:103270007843CDE90021029017A26321C82000F015
:103280008EF9002020214FF6FF724FF47843CDE9EC
:103290000021029015A284210A2000F080F900206C
:1032A00020214FF6FF724FF47843CDE900210290C0
:1032B00011A284214FF4877000F071F90EBD000057
:1032C0000004004864656661756C74004375727231
:1032D000656E74563A0000006D7600004D617856B8
:1032E0003A0000004D696E563A0000004C696E6568
:1032F00061726974793A0000250000002DE9FF5FD2
:1033000080468A4617469B460F9D00200290CDF8C6
:103310000080284605EBD071C1F347042046E21730
:1033200004EB5272D2102146E31704EB5373DB1007
:10333000A4EBC3030BB1012300E000231A446A434A
:1033400092B20192A7F12000C7B20AEB0500401E1D
:1033500083B208EB0400401E82B251464046FFF79C
:1033600032FD002669E00C2D07D107EB47003549F7
:1033700001EB8000805D03901BE0102D05D13248E9
:1033800000EB0710805D039013E0182D07D107EBC9
:1033900047002E4901EB0010805D039009E0202DCD
:1033A00005D12B4800EB8710805D039001E0BDE85C
:1033B000FF9F4FF000093AE01098C8B9012000FAC9
:1033C00009F00399084018B1584600F009F902E0E5
:1033D0000E9800F005F90298401CC0B202900298C5
:1033E00090FBF4F104FB1100E8B90020029021E009
:1033F000012000FA09F00399084020B15A465146CD
:103400004046FFF757FD08F101001FFA80F80098C9
:10341000A8EB0000A04206D1DDF800800AF101000F
:103420001FFA80FA06E009F1010000F0FF09B9F186
:10343000080FC1DB00BF701C86B20198864292DB88
:1034400000BFB4E7985600080C5B0008FC60000859
:10345000CC7200082DE9FF4F2DED020B2DED028BF4
:1034600083B00746B0EE408A1446DDE91486304644
:1034700006EBD071C1F3470A9FED220A28EE000A3D
:10348000BCEEC00A10EE100A1FFA80FB002530E0E7
:10349000601B401EC1B20A2001F0CEFBBBFBF0F066
:1034A0000A21B0FBF1F201FB1209A01EA84210D1C3
:1034B0000020A11E01FB0A71CDE90086029088B2AE
:1034C0002E220A9B0899FFF719FF681CC5B2601CE1
:1034D000C4B2002009F13001CAB205FB0A71CDE97E
:1034E0000086029088B20A9B0899FFF707FF681CC4
:1034F000C5B2A542CCDB03B0BDEC028B06B0BDE883
:10350000F08F00000000C8422DE9FF4F85B007464C
:1035100091461D46DDE913A600200490304606EBD7
:10352000D071C1F3470B002434E0281B401EC1B208
:103530000A2001F081FBB9FBF0F00A21B0FBF1F2A7
:1035400001FB12080498A0B9681EA04211DDB8F171
:10355000000F0CD1002004FB0B71CDE900A60290F6
:1035600088B22022129B0699FFF7C8FE10E00120C6
:103570000490002008F13001CAB204FB0B71CDE9C0
:1035800000A6029088B2129B0699FFF7B7FE00BF13
:10359000601CC4B2AC42C8DB09B0BDE8F08F2DE9B5
:1035A000FE4F06460F4614469846DDE90D5ADDF8F3
:1035B000309010E0CDE9015ACDF8009022784346D2
:1035C00039463046FFF79AFE284605EBD07106EBE8
:1035D00061018EB2641C20780028EBD1BDE8FE8F1B
:1035E00010B50446201200F01DF8E0B200F01AF801
:1035F00010BD10B50446204600F014F810BD10B5FB
:103600000446002204214FF09040FDF707FC2046BD
:1036100000F008F8012204214FF09040FDF7FEFB76
:1036200010BD000070B50446002201214FF090400B
:10363000FDF7F4FB002523E000224FF4005115486C
:10364000FDF7ECFB012000F03DFE04F0800028B106
:103650000122D1030F48FDF7E1FB05E000224FF402
:1036600000410C48FDF7DAFB012251030948FDF740
:10367000D5FB012000F026FE6006040E681CC5B2D2
:10368000082DD9DB012211464FF09040FDF7C6FB13
:1036900070BD0000000400488168024A1140491CC6
:1036A00081607047C0FFFF7F024602F1600000EBBF
:1036B0008103186800F0F840704701468868C0F33D
:1036C000C00070470146886800F00100704701465D
:1036D0008868C0F30070704701468868C0F38000B6
:1036E000704700008168024A1140091D81607047DF
:1036F000C0FFFF7F70B500F11404C1F3406504EB17
:1037000085031C68C1F304560725B540AC43C1F3DB
:10371000045502FA05F52C431C6070BD826822F046
:10372000E0720A438260704710B500F1600404EB58
:1037300081031C6824F0004414431C6010BD4269DE
:1037400022F000420A4342617047000000B587B092
:10375000182101A8FCF78EFD1A481B4908600020BB
:103760004860002118488160C16001610421416105
:103770000021017641760121C161002180F82010ED
:103780008162C16280F83010416380F83810FDF723
:10379000B1F808B1FCF737FE0C4801900620029002
:1037A000032003907F2004900420059000200690C1
:1037B00001A90548FCF72AFE08B1FCF724FE07B072
:1037C00000BD000000000450840000200004002A16
:1037D00000B587B0142102A8FCF74CFD00BF2E48AD
:1037E000C06C40F080002C49C8640846C06C00F0F2
:1037F0008000019000BF00BF00BF0846C06C40F0D1
:103800000100C8640846C06C00F00100019000BFD0
:1038100000BF00BF0846C06C40F00200C864084604
:10382000C06C00F00200019000BF00BF01220D211A
:103830004FF09040FDF7F2FA012211031748FDF70F
:10384000EDFA00224FF4E0711448FDF7E7FA0D207D
:1038500002900120039000200490059002A94FF0EF
:103860009040FDF7F3F940F22320029000200390EE
:10387000049002A90948FDF7E9F94FF48E5002902F
:103880000120039000200490059002A90348FDF751
:10389000DDF907B000BD0000001002400004004840
:1038A00010B51248124908601248486000211048BB
:1038B00081600121C1600021016141618161C161BB
:1038C0000162FDF721FB08B1FCF79DFD00210848CE
:1038D000FDF7B0FA08B1FCF796FD00210448FDF7AA
:1038E000DEFA08B1FCF78FFD10BD00000084004037
:1038F000EC000020EC9C901010B5114811490860B4
:103900004FF48270486000210E4881604FF4E061FE
:10391000C1600021016101214161490281613021C1
:10392000C16100210162416281620721C1620021FF
:1039300001634163FEF7BCFB08B1FCF764FD10BDF9
:10394000003001404001002010B5114811490860C5
:103950004FF48270486000210E4881604FF440713E
:10396000C16002210161012141614902816120217F
:10397000C16100210162416281620721C1620021AF
:1039800001634163FEF794FB08B1FCF73CFD10BDF9
:1039900000380040A401002000B58DB0242104A807
:1039A000FCF768FC00200190029003901848194928
:1039B0000860002048600021164881604FF6FF71C2
:1039C000C1600021016141618161032004900020F8
:1039D0000590012006900020079008900990012092
:1039E0000A9000200B900C9004A90A48FEF7B4FF3F
:1039F00008B1FCF708FD002001900290039001A996
:103A00000448FEF7C3FE08B1FCF7FDFC0DB000BD95
:103A1000002C0140080200200EB50020009001900B
:103A200002900E480E4908604F20486000210C4863
:103A3000816040F2E731C16000218161FEF7F0FE54
:103A400008B1FCF7E0FC00200090029069460448B1
:103A5000FEF79CFE08B1FCF7D6FC0EBD001000403E
:103A60005402002000BFFEE700BFFEE770470000E1
:103A70002DE9F04104460F4600255B48C06800F080
:103A8000030090B15848C06800F0030021688842E4
:103A900009D1206838B15448C068C0F30210401CF6
:103AA0006168884233D0012531E02068012804D0C4
:103AB000022809D003281AD10DE04B48006800F015
:103AC000020000B9012514E04748006800F4806056
:103AD00000B901250DE04448006800F4003028B921
:103AE0004148006800F4802000B9012501E001256B
:103AF00000BF00BF5DB9D4E90010401E41EA0010CC
:103B00003949C96821F0730108433749C860002D5D
:103B100067D13548006820F0806033490860FDF7C0
:103B200083F9064606E0FDF77FF9801B022801D9DC
:103B3000032505E02C48006800F000600028F2D161
:103B400000BFC5BB67B9A0680002217B40EAC16025
:103B500025490969254A114008432349086120E0A5
:103B6000012F0FD1A0680002218A0122C2EB51016E
:103B700040EA41501C4909691D4A114008431A494D
:103B800008610EE0A0680002217D0122C2EB510114
:103B900040EA416014490969164A11400843124934
:103BA00008611148006840F080600F490860FDF727
:103BB0003BF9064607E014E0FDF736F9801B0228C2
:103BC00001D9032505E00848006800F000600028DE
:103BD000F2D000BF2DB904480069A1690843024929
:103BE00008612846BDE8F08100100240FF80FF0711
:103BF000FF809FFFFF80FFF9F8B5044600262348A9
:103C0000806D00F0805018B1FDF74AFB054616E0C4
:103C100000BF1E48806D40F080501C4988650846F2
:103C2000806D00F08050009000BF00BFFDF738FBB2
:103C300005461648806D20F0805014498865B5F51A
:103C4000007F07D1802C10D9A02C01D902260CE0CE
:103C500001260AE0802C01D9032606E0802C01D140
:103C6000022602E0702C00D101260948006820F0ED
:103C700007003043064908600846006800F0070066
:103C8000B04201D00120F8BD0020FCE70010024046
:103C900000200240F8B504460E4615463346002281
:103CA0004FF4C0512046009500F026F828B1206E50
:103CB00040F0200020660320F8BD3346002280211A
:103CC0002046009500F094F828B1206E40F02000C6
:103CD00020660320F0E7334600224FF4C0612046FF
:103CE000009500F009F828B1206E40F02000206611
:103CF0000320E1E70020DFE72DE9FC5F04460D46E5
:103D000016461F46DDF8309000200090FDF78CF835
:103D1000A0EB0900A7EB0008FDF786F882462068B3
:103D200000F10C0B31480068C0EBC00000EB8000D4
:103D3000000D00FB08F0019050E0B5F5C06F05D113
:103D400026B99BF8000000909DF80000781C002820
:103D500044D0FDF769F8A0EB0A00404502D2B8F163
:103D6000000F34D12068406820F0E00021684860EE
:103D70006068B0F5827F0DD1A068B0F5004F03D028
:103D8000A068B0F5806F05D12068006820F0400081
:103D900021680860A06AB0F5005F0DD100BF2068FF
:103DA000006820F40050216808602068006840F432
:103DB00000502168086000BF012084F85D0000BF4A
:103DC000002084F85C0000BF0320BDE8FC9F019840
:103DD00008B94FF000080198401E019020688068E3
:103DE0002840B042A9D10020EFE700000C000020DD
:103DF0002DE9F84F04460D4690461E46DDF8289002
:103E0000FDF712F8A0EB0900371AFDF70DF882460E
:103E10002C480068C0F3CB307843009045E0701C1C
:103E2000002842D0FDF700F8A0EB0A00B84200D20B
:103E3000A7BB2068406820F0E00021684860606807
:103E4000B0F5827F0DD1A068B0F5004F03D0A06817
:103E5000B0F5806F05D12068006820F0400021682F
:103E60000860A06AB0F5005F0DD100BF206800684F
:103E700020F40050216808602068006840F4005079
:103E80002168086000BF012084F85D0000BF0020A9
:103E900084F85C0000BF0320BDE8F88FFFE70098BE
:103EA00000B900270098401E0090206880682840D4
:103EB000A84201D1012000E000204045AFD1002000
:103EC000EAE700000C000020704710B5FDF7D4F8B9
:103ED00010BD00B597B0442106A8FCF7CBF914211A
:103EE00001A8FCF7C7F94FF40070FDF793F908B18A
:103EF000FCF789FA01200690000407900220109038
:103F00000321119101211291142113910721149180
:103F100002211591169106A8FDF722FD08B1FCF7C4
:103F200072FA0F2001900320029000200390049069
:103F30000590042101A8FDF7C3FB08B1FCF763FA63
:103F400017B000BD0348006840F4700001490860E4
:103F50007047000088ED00E010B50248FEF705FE4E
:103F600010BD00005402002010B502681F4B98429B
:103F700005D0B0F1804F02D01D4B984203D122F002
:103F800070024B681A43194B98420BD0B0F1804F26
:103F900008D0174B984205D0164B984202D0164BCA
:103FA000984203D122F44072CB681A4322F0800376
:103FB0004C6943EA040202608B68C3620B68836247
:103FC0000A4B984205D00B4B984202D00A4B9842BC
:103FD00001D10B69036301234361036903F001030A
:103FE0001BB1036923F00103036110BD002C0140E4
:103FF00000040040004001400044014030B501F0A1
:104000001F05012404FA05F3046A9C430462046A50
:1040100001F01F0502FA05F52C43046230BD00BF14
:10402000FEE7000002480068C0F30220704700006D
:104030000CED00E010B5002804DB0A07130E054A5A
:10404000135406E00A07140E034A00F00F031B1F67
:10405000D45410BD00E400E018ED00E02DED020B9B
:10406000019820F0004001909DED000B02B07047D8
:1040700010B52DED068B2948FCF738FC284908803F
:104080000846008801F0A2F841EC1A0B9FED250BC1
:1040900053EC102B00F0CEFE41EC190B9FED230BDF
:1040A00053EC102B01F0E2F841EC180B00F0DCFDB2
:1040B000204908601948FCF76BFD1E4890ED000A86
:1040C000BCEEC00A10EE100A1B491C4A126841F8E7
:1040D000220008461949096850F821001849096862
:1040E00008441749086015480068401C13490860D7
:1040F00008460068B0F57A7F0CDB114800684FF481
:104100007A71B0FBF1F00F49086000200C4908609B
:104110000A490860BDEC068B10BD00008400002039
:104120004C000020000000000000B0400000000033
:1041300000C8A94050000020A42200205400002004
:1041400044000020480000201FB53A200390C420FE
:104150000290982001900020009000224FF480717E
:104160001748FCF75BFE062000F074F80A2000F008
:10417000A3F8012211021248FCF750FE03AA012104
:10418000002000F071F802AA0121084600F06CF846
:1041900001AA0121022000F067F86A4601210320EC
:1041A00000F062F800224FF480710548FCF736FEFB
:1041B0000A2000F081F8082000F04CF81FBD000034
:1041C0000004004810B500224FF480711648FCF737
:1041D00025FE102000F03EF800F02AF81349086090
:1041E00000F026F81149096840EA01200F490860EB
:1041F00000F01EF80D49096840EA01200B490860EB
:104200000846006800F4000030B1084600686FF00E
:104210007F41401A05490860012211020248FCF75B
:10422000FDFD0248006810BD000400482800002081
:104230000EB5FF200290002001900A20012301AA60
:1042400002A900900248FEF716F99DF804000EBD81
:104250004001002001B50A23012269460148FEF70A
:104260000DF808BD400100202DE9F04106460C463E
:10427000154600224FF480710E48FCF7CFFD0C214B
:1042800001EA8601621E02F00302114341F0400080
:10429000FFF7E0FF002704E015F8010BFFF7DAFF56
:1042A0007F1CA742F8DB012211020248FCF7B6FD91
:1042B000BDE8F0810004004801B50098FCF7B2FCAD
:1042C00008BD000011B526E0009CB4F5617F02D95D
:1042D0004FF4617400E0009C23464FF0E024A06995
:1042E000502404FB1301002908DB00BF4FF0E02439
:1042F000A26982420CDA8A42F8DA09E0084C2144C9
:1043000000BF4FF0E024A2698242FADD8A42F8DC65
:10431000009CE41A0094009C002CD5D118BD00002C
:104320008038010010B52DED068BFFF74BFF0446DA
:1043300000F035FF41EC1A0B9FED330B53EC102BC3
:1043400000F094FF41EC190B9FED310B53EC102B57
:1043500000F070FD41EC180B00F0C4FE2E4908601F
:104360002E48006801284CD12D4800680968884211
:1043700020DA294800682A4908602A490968A1F515
:104380001C50103800F00BFF41EC1A0B9FED260B70
:1043900053EC102B00F04EFD41EC190B9FED240B5C
:1043A00053EC102B00F062FF41EC180B00F09AFE6A
:1043B000214908602148006817490968884220DDC2
:1043C000154800681D49086016490968A1F51C5088
:1043D000103800F0E4FE41EC1A0B9FED130B53EC88
:1043E000102B00F027FD41EC190B9FED110B53EC46
:1043F000102B00F03BFF41EC180B00F073FE10494E
:104400000860BDEC068B10BD0000000000C8A9408C
:104410000000000000006041100000202400002087
:10442000140000203C0000200000000000808640B6
:104430000000000000C06F40180000201C00002099
:104440002000002010B52DED0A8B9FED3E0BB0EE45
:10445000408AF0EE608A00F01FFB00F085FB00242C
:104460004BE03A4951F8240000F099FE41EC1C0B56
:10447000374800EBC40090ED001BB0EE410AF0EEAF
:10448000610A53EC102B51EC1C0B00F0EDFF41ECDA
:104490001B0BB0EE4B0AF0EE6B0AFFF7DFFDB0EE40
:1044A000409AF0EE609AB0EE480AF0EE680AFFF724
:1044B000D5FDB0EE40AAF0EE60AA53EC192B51ECFA
:1044C0001A0B00F097FE17D2204951F8240000F093
:1044D00066FE41EC190B1E4800EBC40090ED001B7A
:1044E000B0EE410AF0EE610A53EC102B51EC190BBF
:1044F00000F0BAFF41EC180B641C164800688442B7
:10450000AFDB14490968491E104A52F8211012689D
:10451000881A00F044FE41EC1A0B53EC1A2B51ECB4
:10452000180B00F087FC41EC190BB0EE490AF0EED5
:10453000690AFFF793FD084880ED000BBDEC0A8B7C
:1045400010BD000000000000000000004832002004
:10455000485200205800002070000020FEB590480E
:104560000068022835D18F48006890BB42F2107075
:104570008D490968486200208C4908604FF48061C9
:104580008B48FBF777FE4FF480618A48FBF772FE99
:10459000002020214FF6FF724FF47843CDE900212F
:1045A000029085A201460A20FEF7F9FF01207D490D
:1045B0000860834883490860002083490860804878
:1045C00040428249086000208149086000218148FA
:1045D00001607348006803287ED172480068012892
:1045E000FAD100206F49086020214FF6FF724FF486
:1045F0007843CDE90021029077A201460A20FEF718
:10460000CEFF71490968724A1268881A002801DBD6
:10461000014600E04142B1F5FA7F03DA012070491A
:10462000086026E068490968694A1268881A002803
:1046300001DB014600E0414240F24C42914203DA84
:1046400002206749086014E05F490968604A1268FF
:10465000881A002801DB014600E0414240F634029E
:10466000914203DA03205E49086002E004205C49BD
:10467000086042F20F74002015E05A4A52F82010E8
:10468000002901DB0A4600E04A42A2420ADC554A00
:1046900052F82010002901DB0A4600E04A42144685
:1046A00051490860401C4B4909688142E5DC0025FE
:1046B00000264B48006801280FD14C484A49096838
:1046C00050F82100A0F5B17548484749096850F8ED
:1046D000210000F5B17638E060E04148006802282A
:1046E0000ED142484049096850F82100A0F53175C3
:1046F0003E483D49096850F8210000F5317624E034
:104700003748006803280ED138483749096850F8FF
:104710002100A0F2176535483349096850F8210097
:1047200000F2176611E02E48006804280DD12F48CA
:104730002D49096850F82100A0F53A652B482A490F
:10474000096850F8210000F53A6600201FE027496B
:1047500051F82010A94219DB244951F82010B14228
:1047600014DC204951F82010114A104B1B6842F804
:1047700023101E4951F820200E490C4B1B6841F8AC
:1047800023200A490968491C084A1160401C114944
:1047900009688142DBDCFFF755FE00BFFEBD00006B
:1047A000780000202400002008020020580000208B
:1047B000483200204842002074657374696E6700B7
:1047C000C1BDF0FF14000020180000201C000020D4
:1047D00020000020A0220020726561647920200062
:1047E0007C000020A002002080000020A0120020F9
:1047F00030B52DED0A8B83B09348056800249348AB
:10480000006800F0E3FC41EC1C0B9FED910B53ECB6
:10481000102B00F029FE41EC1B0B9FED8F0B53EC8E
:10482000102B00F007FB41EC1A0B9FED8D0B53ECA6
:10483000102B00F01BFD41EC190B9FED8B0B53EC83
:10484000102B00F043FA41EC180B00F07BFC84B213
:10485000B4F5937F01DD4FF49374D82C00DAD8249B
:10486000ED2C13DD4FF4FC601D2322460621009041
:10487000D820FEF752FB4FF6FF701D234FF49372C2
:10488000062100902046FEF748FB12E04FF6E0704C
:104890001D23224606210090D820FEF73EFB4FF64E
:1048A000FF701D234FF49372062100902046FEF7FF
:1048B00034FB002D11DA002020214FF6FF724FF457
:1048C0007843CDE90021029069A22121A520FEF7BD
:1048D00066FE6842674908600FE0002020214FF61D
:1048E000FF724FF47843CDE90021029062A22121AA
:1048F000A520FEF754FE5F48056020204FF6FF71AB
:104900004FF47842CDE9002102905A48008882B2E3
:1049100004232121B420FEF7F7FD58480068002841
:1049200013DA002020214FF6FF724FF47843CDE9CF
:10493000002102904EA242216920FEF730FE4F482E
:10494000006840424E49086011E0002020214FF6E7
:10495000FF724FF47843CDE90021029046A2422134
:104960006920FEF71CFE4548006845490860202084
:104970004FF6FF714FF47842CDE900210290404894
:10498000008882B2042342217820FEF7BDFD3D4815
:104990000068002813DA002020214FF6FF724FF440
:1049A0007843CDE90021029031A263216920FEF70E
:1049B000F6FD3448006840423349086011E00020A9
:1049C00020214FF6FF724FF47843CDE90021029089
:1049D00029A263216920FEF7E2FD2A4800682A49DE
:1049E000086020204FF6FF714FF47842CDE9002196
:1049F00002902548008882B2042363217820FEF7C4
:104A000083FD9FED220B53EC102B224890ED000B01
:104A100051EC100B00F02AFC41EC190B00F024F9CA
:104A200008EE100A20204FF6FF714FF4784304225D
:104A3000B0EE480ACDE900108421B420FEF70AFD4B
:104A400003B0BDEC0A8B30BD1000002048000020F0
:104A50000000000000C0924000000000008066409E
:104A600000000000000051400000000000006B400A
:104A70002D0000002C0000202B000000140000205E
:104A8000300000201C000020340000200000000046
:104A9000000059407000002070B52DED088B9FED8F
:104AA0002B0BB0EE409AF0EE609A9FED280BB0EE23
:104AB000408AF0EE608A9FED250BB0EE40AAF0EE42
:104AC00060AA24480468611E234A52F82110126823
:104AD000881A00F064FB41EC190B20490A68611E3A
:104AE0001E4B53F82110501A00F059FB41EC180BE3
:104AF000611E1A4A52F82110174A12685143174A88
:104B00001368621E144D55F8222003FB121000F0AA
:104B100046FB41EC1A0B53EC182B51EC190B00F02F
:104B200089F941EC1B0B00F092F80D4A03C253ECDB
:104B3000182B51EC1A0B00F07DF941EC1B0B00F027
:104B400086F8084A03C2BDEC088B70BD0000000067
:104B50000000000058000020483200204842002099
:104B6000600000206800002010B52DED048B0024AB
:104B70001FE0134951F8240000F011FB41EC190B20
:104B8000104890ED000B53EC102B51EC190B00F07A
:104B90006DFB41EC180B0C4890ED000B53EC102B07
:104BA00051EC180B00F092F8084A02EBC40203C261
:104BB000641C074800688442DBDBBDEC048B10BD3D
:104BC0004842002060000020680000204852002079
:104BD00058000020FCF75CFAFFF77BF9FEF7F8FDC0
:104BE000FEF7B4FDFEF75CFEFEF786FEFEF7ACFEB8
:104BF000FEF7D2FEFEF710FF0C48FBF7C9FF0C488A
:104C0000FDF768FE04210B48FDF748FF42F21070E3
:104C1000084909684862FFF797FAFEF7CBF903E005
:104C2000FFF79CFCFFF7E4FDFAE70000840000209A
:104C3000540200200802002010B50246012000E0C6
:104C400050430B00A1F10104E1B2F9D110BD81F094
:104C50000041704780F00040704721F000417047EC
:104C600020F000407047000021F00042A2F16052A5
:104C7000B2F5801F01F0004328BFD2F17F6C0BD941
:104C80005FEA001C43EAC20242EB507018BF704753
:104C900028BF20F001007047B2F5801FBCBF184646
:104CA00070474FEA410C1CF5001F02D2084600F085
:104CB000CABC70B500F084FB00000089FFF7F6BFA6
:104CC0004FF00040A0F580007047000010B591EA59
:104CD000030F48BF83F0004300F1CE83841A71EBC9
:104CE000030C05D2121943EB0C03001B61EB0C0102
:104CF000DFF824E14FEA1154A4EB135C1EEA430FE2
:104D000018BF9EEA445F73D023EA0E03DCF1200E45
:104D100021EA045143F4801332D322FA0CFE10EB43
:104D20000E0023FA0CFE41EB0E01CCF1200E03FA2B
:104D30000EFE10EB0E0051F10001B1F5801FCCF119
:104D4000200E32D201EB045112FA0EF2BDE81040EF
:104D500058BF7047401C38BF5FEA420218BF704717
:104D6000002814BF20F0010041F100014FEA410387
:104D700013F5001F38BF7047A1F1C04100F06EBBB2
:104D8000012A43EB0302ACF1200CDCF11F0E32BF11
:104D90004FF0000E23FA0CF310EB030041EB04512B
:104DA000B4EB115FD0D0A1EB045101F5801149089B
:104DB0005FEA300001EB04510ED350F1000038BF20
:104DC00012FA0EFE08D1BDE81040C9E7401C38BFFA
:104DD0005FEA4202CAD1C3E7BDE810404FEA41038F
:104DE00013F5001F38BF7047A1F1C04100F036BB7A
:104DF0009EEA445F08D011EA5E0FBDE8104004BF90
:104E000001F0004100207047BDE8104070B500F08F
:104E1000D7FA00BF64FBBE3E0000E0FF491058BF58
:104E2000C1F140415B1058BFC3F140438B42EFF3E7
:104E3000008070472DE9C04130B4DFF8A0C23CEAE1
:104E4000111418BF3CEA131400F0EC8081EA03054A
:104E50001CEA111444EAD57418BF1CEA131500F0BB
:104E6000C780A4EB05044FF0004545EAC12145EA9F
:104E7000C32341EA505143EA525304F17F749942EB
:104E800004F500344FEAC0204FEAC22208BF904226
:104E900000F09C804FEA13650FF24016765D4FEAF2
:104EA000134506FB05F7C7F1807706FB07F74FEAC6
:104EB000D737A7FB03687642C8F58038A7FB06CE34
:104EC00038BFA8F1010807FB08E64FF0000EA6FB6B
:104ED000028CE6FB03CEDCF1000CCEF1004E38BFB5
:104EE000AEF1010EA6FB0C584FF000074FF0000585
:104EF000E6FB0E87A1FB08C6A0FB07CE16EB0E064D
:104F000045F10005E1FB076515F1E04E7EBFA4F514
:104F100080345FEA46066D4116F1800745F10005D1
:104F20004FEA17274FEA066647EA0567A6F1DE460D
:104F3000B6F1805F4FEA15251FD9384624F0010CE1
:104F400005EBC471BCF1FE6F01EB0C1102D8F0BC93
:104F5000BDE8008124425CBF01F5801E9EEAC47F4B
:104F600002D4F0BCBDE80081244238D4F0BCA1F1E9
:104F7000C041BDE8004100F071BA4FEAD22242EAD6
:104F800043524FEAD323A7FB02864FEAD02040EAE0
:104F9000415007FB03661EEA0E0F4FEAD12105FBC5
:104FA000026658BFA6EB0056B6EB00564FEA520E0B
:104FB0004EEAC37E18EB0E0E56EB530EBDD518EB22
:104FC00002085E417F1C55F10005B6E74FF48015DD
:104FD0004FF000074FF000064FF00008ADE7F0BCBF
:104FE0004FF0000001F1C04101F00041BDE8008137
:104FF00011EA0C1F0CEA131500D00CE013EA0C1F89
:1050000000F025804FF00000F0BC81EA030101F0C0
:105010000041BDE80081F0BCBDE8004181EA030128
:1050200000F01CBAF0BCBDE8004170B500F0C8F952
:10503000097EFC3E00F007B881EA03014FF0000052
:1050400001F00041704781EA030100F007BAF0BCAB
:10505000BDE800414FF0000021497047FFFDFBF91A
:10506000F7F5F4F2F0EEEDEBE9E8E6E4E3E1E0DE9B
:10507000DDDBDAD8D7D5D4D3D1D0CFCDCCCBCAC80D
:10508000C7C6C5C4C2C1C0BFBEBDBCBBBAB9B8B734
:10509000B6B5B4B3B2B1B0AFAEADACABAAA9A8A827
:1050A000A7A6A5A4A3A3A2A1A09F9F9E9D9C9C9BF5
:1050B0009A999998979796959594939392919190A0
:1050C0008F8F8E8E8D8C8C8B8B8A89898888878731
:1050D0008685858484838382828181800000FF07A6
:1050E0000000F87F4FEA41034FEA5353A3F5806372
:1050F000D3F11E03C8BFD3F1210C0CDD4FF00042E9
:1051000042EAC12242EA505232FA03FC8CEAE17CC4
:10511000ACEBE1707047102BC4BF0020704703F563
:10512000787CBCF1FF3F04D06FF0004282EA21009E
:10513000704770B500F044F9499224800020704710
:10514000F2E700004FEA1153A3F58063D3F11E0389
:10515000A8BFD3F1200C08DB4FF0004242EAC12285
:1051600052EA505232FA03F0704709420BD4102B26
:10517000C4BF0020704703F5787CBCF1FF3F05D029
:105180004FF0FF3070474FF00000704770B500F0EF
:1051900017F900BF4992248000207047F0E710F013
:1051A000004248BF4042B0FA80F310FA03F10AD03F
:1051B000C3F11D0303F580634FEA415002EB035234
:1051C00002EBD12170474FF000007047B0FA80F336
:1051D00010FA03F10AD0C3F11D0303F580634FEA0F
:1051E00041504FEA035202EBD12170474FF00000CB
:1051F0007047000051EA030C17D41CF5801F58BFFC
:10520000BCF5801F00F10680994218BF704708BFA7
:105210009042704707D711F5801F58BF13F5801FC4
:1052200019D499427047894270471CF5801F08D5F0
:10523000BCF5801FF7D58B4218BF704708BF82426C
:1052400070474FF4001C1CEB410F38BF1CEB430FA1
:1052500001D28B42704770B500F0B2F89224490039
:105260004FF000514FF08053FFF7D8BDDFF848C131
:1052700070B51CEA111E1EBF1CEA13159EEA0C0F26
:1052800095EA0C0F00F06F8081EA030423EA4C13C7
:105290004EEAD47E21EA4C1141F4801143F480138C
:1052A000AE44A1FB024CA0FB0365AEF17F7E361934
:1052B00055EB0C05A1FB034C4CF10003A0FB021CB9
:1052C00016EB0C06654153F10003094218BF46F086
:1052D000010613F4007F0BD14FEA03314FEA05308A
:1052E000340341EA155140EA16506FF003020AE018
:1052F0004FEAC3214FEAC520F40241EA555140EA82
:1053000056506FF0020202EB2E4201EB025585EA85
:10531000CE710AD05FEA440C18BF24F0004450F16B
:10532000000041F1000120EAD47040F2FE7C6245A9
:1053300000D270BDA84214BF4FF080444FF04044EB
:10534000002E08BF0024BEF1806FA8BFA1F1C041AC
:10535000BDE8704080F282804FF0000001F1C04152
:1053600001F0004170479EEA0C0F0CEA131518BFBC
:1053700095EA0C0F06D04FF0000081EA030E0EF004
:10538000004170BD00F01CF88900013E00F007B834
:1053900000F009B84FEA430C5FEA5C5C08D081EA90
:1053A000030100F05BB84FEA410C5FEA5C5CF6D1A8
:1053B0004FF00000014970470000FF070000F87F30
:1053C0000EF1020E2EF0030E5EF8046B364205D489
:1053D000012A43EB030515F5001F12D8012841EB04
:1053E000010C1CF5001F0CD80ED14FEAD17C15F52D
:1053F000001F0CEB4C0C0CF1020C08BF4CEBD37CE7
:1054000004E04FF0080C01E04FEAD37C0CEB4C05B4
:1054100026FA05F606F00706B6F1040C06D20EEBE6
:10542000860CBDE870404CF0010C6047DFE80CF0E2
:10543000090B02024FF000414FF00000A1F50021DE
:1054400070BD19461046012851EB010418BFD4F570
:10545000001484BF002001F0004170BD0808A0F5D1
:1054600000114FEA3101704710B591EA030F48BFB0
:1054700083F000433FF532AC841A71EB030C07D282
:1054800012198CF0004C43EB0C03001B61EB0C0178
:10549000DFF8A4E14FEA1154A4EB135C1EEA430FBA
:1054A00018BF9EEA445F00F0B08023EA6E035242C8
:1054B00021EA0451C3EB6E0338BF5B1EDCF1200E02
:1054C00025D322FA0CFE10EB0E0043FA0CFE41EB42
:1054D0000E01CCF1200E03FA0EFE10EB0E0051F17E
:1054E0000001CCF1200E29D412FA0EF201EB045186
:1054F000BDE8104058BF7047401C1CBFB2F1004FC0
:10550000704700280CBF491C20F00100704712EBC7
:10551000020E43EB030218BF4FF0010E4EEA4202A7
:10552000ACF1200CDCF11E0E54D943FA0CFE10EB4A
:105530000E0051F1FF31CCF11E0ED5D50EF1010E4A
:1055400012FA0EFE404141EB010101EB445C5FEABF
:105550005C5C10D910EBDE7001EB045138BFBEF17A
:10556000004FBDE8104018BF704700280CBF491C11
:1055700020F00100704730D24FEAD42C11F5001111
:1055800024F400641BD0B1FA81F20B3AA41AA41ED1
:10559000D2F12003914030FA03F31943904001EB1C
:1055A000CC71002C01EB0451BDE81040A8BF70473E
:1055B00001F1C0414FF0000001F000417047B0FA26
:1055C00080F310FA03F100D110BDE41A173C48052E
:1055D000C90AE4E701EB045110BD491001EB045185
:1055E000BDE810404FEA300002E04FF00001704784
:1055F0004A0008BF0042F8D0B2F5001F28BF70472C
:1056000001F000414FF0000070479EEA445F07D070
:1056100011EA5E0FBDE8104004BF00210020704772
:10562000BDE8104070B5FFF7CBFE00BF40DFF63E8F
:1056300083F00041104670470000E0FF4FF04070DB
:10564000E1EE100A7047FF2141EAD050C0057047D3
:105650000000000000000000010203040607080922
:105660000000000001020304A0860100400D0300B9
:10567000801A060000350C0040420F0080841E0096
:1056800000093D0000127A000024F40000366E018B
:105690000048E801006CDC0200000000000000008F
:1056A00000000000000004040404040000040000E2
:1056B00014140A00000000000000000000000A0AA4
:1056C0001F0A0A1F0A0A000000040E1505060C1422
:1056D000150E0400000012150D152E2C2A120000C4
:1056E0000000040A0A3615152916000002020100FE
:1056F0000000000000000000100808040404040476
:10570000080810000204040808080808040402003D
:1057100000000004150E0E15040000000000000833
:10572000083E080800000000000000000000000023
:105730000202010000000000003F00000000000025
:105740000000000000000000000200000020101017
:10575000080804040202010000000E1111111111C9
:10576000110E00000000040604040404040E0000EE
:1057700000000E1111080402011F000000000E11AC
:10578000100C1010110E00000000080C0C0A091F6C
:10579000081C000000001F01010F1110110E000075
:1057A00000000C12010D1311110E000000001E105C
:1057B000080804040404000000000E11110E111169
:1057C000110E000000000E1111191610090600003C
:1057D00000000000040000000004000000000000C1
:1057E0000004000000040400000010080402020489
:1057F00008100000000000003F003F000000000013
:1058000000000204081010080402000000000E113D
:10581000110804040004000000001C22292D2D1D85
:10582000221C0000000004040C0A0A1E12330000AF
:1058300000000F12120E1212120F000000001E11B3
:1058400001010101110E000000000F1212121212CC
:10585000120F000000001F120A0E0A02121F0000A1
:1058600000001F120A0E0A020207000000001C12AC
:1058700001013911120C000000003312121E121225
:105880001233000000001F0404040404041F00007D
:1058900000003E0808080808080809070000371239
:1058A0000A060A1212370000000007020202020272
:1058B000223F000000003B1B1B1B15151535000087
:1058C00000003B1216161A1A1217000000000E11E3
:1058D00011111111110E000000000F12120E020220
:1058E0000207000000000E1111111117190E180007
:1058F00000000F12120E0A121237000000001E11D3
:1059000001060810110F000000001F150404040414
:10591000040E00000000331212121212120C0000CA
:1059200000003312120A0A0C0404000000001515CE
:1059300015150E0A0A0A000000001B0A0A04040AD0
:105940000A1B000000001B0A0A0A0404040E0000DF
:1059500000001F0908040402121F00001C040404B4
:105960000404040404041C000002020404040808E3
:10597000081010000E0808080808080808080E009B
:10598000040A000000000000000000000000000009
:10599000000000000000003F0204000000000000C2
:1059A0000000000000000000000C121C123C00006F
:1059B00000030202020E1212120E0000000000008C
:1059C000001C1202120C000000181010101C121201
:1059D000123C000000000000000C121E021C00001F
:1059E00000182404041E0404041E0000000000002B
:1059F000003C120C021C221C00030202020E1212B6
:105A0000123700000004040000060404040E000025
:105A100000080800000C0808080808070003020234
:105A2000021A0A060A13000000070404040404040E
:105A3000041F000000000000000F151515150000E0
:105A400000000000000F12121237000000000000DA
:105A5000000C1212120C000000000000000F1212C5
:105A6000120E020700000000001C1212121C103857
:105A700000000000001B06020207000000000000FA
:105A8000001E020C101E000000000004041E04048E
:105A9000041C000000000000001B1212123C000059
:105AA00000000000001B0A0A0404000000000000BF
:105AB0000015150E0A0A000000000000001B0A0471
:105AC0000A1B000000000000003312120C0804033F
:105AD00000000000001E0804041E0000180808084A
:105AE000080C08080808180008080808080808082A
:105AF0000808080806040404040804040404060052
:105B00001609000000000000000000000000000076
:105B1000000000000000000000000000000000087D
:105B200008080808080800001818000000486C243D
:105B3000120000000000000000000000000000242F
:105B400024247F1212127F12121200000000081C7F
:105B50002A2A0A0C1828282A2A1C080800000022D1
:105B6000251515152A585454542200000000000C25
:105B70001212120A76252911916E00000006060401
:105B800003000000000000000000000000402010A2
:105B90001008080808080810102040000002040837
:105BA0000810101010101008080402000000000077
:105BB00008086B1C1C6B08080000000000000000B7
:105BC000080808087F080808080000000000000016
:105BD00000000000000000000606040300000000B2
:105BE00000000000FE0000000000000000000000B7
:105BF00000000000000000000606000000008040D9
:105C000040202010100808040402020000000018C0
:105C1000244242424242424224180000000000084E
:105C20000E08080808080808083E00000000003CAC
:105C30004242422020100804427E00000000003C46
:105C40004242201820404042221C00000000002058
:105C50003028242422227E20207800000000007EAC
:105C60000202021A26404042221C000000000038B6
:105C70002402021A26424242241800000000007E3C
:105C80002222101008080808080800000000003C44
:105C90004242422418244242423C000000000018C4
:105CA0002442424264584040241C0000000000008E
:105CB0000000181800000000181800000000000084
:105CC0000000000800000000000808040000004078
:105CD000201008040204081020400000000000000A
:105CE00000007F0000007F000000000000000002B4
:105CF0000408102040201008040200000000003CAE
:105D00004242464020101000181800000000001CFD
:105D1000225A555555552D42221C000000000008FE
:105D200008181414243C224242E700000000001F1F
:105D30002222221E22424242221F00000000007C3A
:105D40004242010101010142221C00000000001F2B
:105D50002242424242424242221F00000000003FD3
:105D60004212121E12120242423F00000000003F87
:105D70004212121E12120202020700000000003C32
:105D80002222010101712122221C0000000000E7F3
:105D9000424242427E42424242E700000000003E50
:105DA0000808080808080808083E00000000007CF1
:105DB00010101010101010101010110F00000077AC
:105DC00022120A0E0A121222227700000000000797
:105DD0000202020202020202427F0000000000777B
:105DE000363636362A2A2A2A2A6B0000000000E3BB
:105DF00046464A4A52525262624700000000001C66
:105E00002241414141414141221C00000000003F2C
:105E1000424242423E020202020700000000001C11
:105E20002241414141414D53321C60000000003F7E
:105E30004242423E1212222242C700000000007C71
:105E40004242020418204042423E00000000007F0F
:105E50004908080808080808081C0000000000E7B6
:105E60004242424242424242423C0000000000E7BD
:105E70004242222424141418080800000000006B79
:105E8000494949495555362222220000000000E7C1
:105E9000422424181818242442E700000000007748
:105EA0002222141408080808081C00000000007EC4
:105EB0002120101008040442423F00000078080826
:105EC0000808080808080808080878000000020206
:105ED000040408080810102020204040001E101064
:105EE000101010101010101010101E000038440078
:105EF00000000000000000000000000000000000A2
:105F00000000000000000000000000FF0006080084
:105F10000000000000000000000000000000000081
:105F20000000003C4278444242FC000000000003B4
:105F30000202021A26424242261A00000000000015
:105F400000000038440202024438000000000060F3
:105F5000404040784442424264D8000000000000C3
:105F60000000003C427E0202423C0000000000F0C3
:105F70008808087E08080808083E000000000000A5
:105F80000000007C22221C023C42423C0000000334
:105F90000202023A4642424242E700000000000C80
:105FA0000C00000E08080808083E00000000003041
:105FB00030000038202020202020221E0000000376
:105FC00002020272120A1612227700000000000E6E
:105FD0000808080808080808083E0000000000003B
:105FE0000000007F9292929292B7000000000000A1
:105FF0000000003B4642424242E700000000000031
:106000000000003C42424242423C000000000000CE
:106010000000001B26424242221E02070000000030
:106020000000007844424242447840E00000000012
:10603000000000774C040404041F0000000000006E
:106040000000007C42023C40423E00000000000094
:106050000008083E0808080808300000000000009A
:10606000000000634242424262DC00000000000087
:10607000000000E74224241408080000000000008B
:10608000000000EB494955552222000000000000A5
:106090000000007624181818246E0000000000008C
:1060A000000000E74224241418080807000000003C
:1060B0000000007E22100808447E000000C020205E
:1060C00020202010202020202020C00010101010A0
:1060D00010101010101010101010101000060808EA
:1060E0000808081008080808080806000C32C20052
:1060F00000000000000000000000000000000000A0
:10610000000000000000000000000000000000008F
:10611000000000000000000000000000000000007F
:10612000000000000000000000000000000000006F
:10613000000000006000600060006000600060001F
:10614000600040002000200020000000000000004F
:10615000600060006000000000000000000000001F
:1061600060066006300398018800440000000000CB
:10617000000000000000000000000000000000001F
:10618000000000000000000000000000000000000F
:10619000000000001002100210021002FE07FE07AD
:1061A00008020801080108010801FE07FE070401B2
:1061B00004010401040100000000000000000000D0
:1061C000000040004000F00158034C03CC034C0099
:1061D00058007000E000C001C00140034C035C03A4
:1061E0004C034801F00040004000000000000000A7
:1061F000000000000E010A01910091009100510081
:1062000051003A00AE03A002500450044804480470
:106210004804840284030000000000000000000025
:106220000000000038006C006C006C006C006C001A
:106230002C0098071C011A01330133016301E300AC
:10624000C308C6093C070000000000000000000071
:106250000C001C00100010000800040000000000EA
:10626000000000000000000000000000000000002E
:10627000000000000000000000000000000000001E
:106280000004000200018000800040004000200067
:1062900020002000200020002000200040004000BE
:1062A00080008000000100020004000000000000E7
:1062B0000200040008001000100020002000400030
:1062C000400040004000400040004000200020000E
:1062D0001000100008000400020000000000000090
:1062E00000000000000000004000C0004000460C1C
:1062F0004E0FD001F0015E0F460C40004000400000
:10630000000000000000000000000000000000008D
:1063100000000000000000000000400040004000BD
:1063200040004000FE0F40004000400040004000A0
:10633000000000000000000000000000000000005D
:10634000000000000000000000000000000000004D
:10635000000000000000000000000000000000003D
:106360000C001C00100010000800040000000000D9
:10637000000000000000000000000000000000001D
:1063800000000000FE070000000000000000000008
:1063900000000000000000000000000000000000FD
:1063A00000000000000000000000000000000000ED
:1063B00000000000000000000000000000000000DD
:1063C0001C001C001C000000000000000000000079
:1063D00000040006000200030001000180008000AC
:1063E0004000400060002000200010001000080065
:1063F00008000C000400060002000000000000007D
:10640000000000000000F00098010C030C030606D9
:1064100006060606060606060606060606060C0319
:106420000C039801F00000000000000000000000D4
:1064300000000000000040007C0060006000600080
:10644000600060006000600060006000600060004C
:1064500060006000FC03000000000000000000007D
:10646000000000000000F800840102030603060398
:10647000000300018001C00060002000100008023D
:1064800004020602FE0300000000000000000000FD
:106490000000000000007800C6008601860180012F
:1064A0008001C000700080010001000300030603AA
:1064B00006038601F8000000000000000000000054
:1064C00000000000000080018001C001A001A001C7
:1064D00090018801880184018201FE0F8001800102
:1064E00080018001E00700000000000000000000C3
:1064F000000000000000FC0304000400040004008D
:106500000400F4008C0104030003000306030603E7
:1065100082018401F800000000000000000000007B
:10652000000000000000E00118030C030C00040050
:106530000600E60116030E06060606060606040613
:106540000C021803F0000000000000000000000032
:10655000000000000000F8070C060402040100011E
:1065600000018000800040004000400060006000AA
:1065700060006000600000000000000000000000FB
:10658000000000000000F8010C03060606060606DF
:106590000C021C03F000C8010C03060606060606E2
:1065A00006060C03F00100000000000000000000DF
:1065B000000000000000F0000C010C0306020606BB
:1065C0000606060606078C0678060006000300038A
:1065D0000C018C01780000000000000000000000A9
:1065E00000000000000000000000000000000000AB
:1065F000E000E000E00000000000000000000000FB
:10660000E000E000E00000000000000000000000EA
:10661000000000000000000000000000000000007A
:1066200060006000000000000000000000000000AA
:10663000000060006000400020002000000000001A
:106640000000000000040002000180004000200063
:106650001000080004000800100020004000800026
:106660000001000200040000000000000000000023
:10667000000000000000000000000000000000001A
:10668000FE07000000000000FE0700000000000000
:1066900000000000000000000000000000000000FA
:1066A00000000000040008001000200040008000EE
:1066B00000010002000400020001800040002000F0
:1066C00010000800040000000000000000000000AE
:1066D000000000000000E0031806040C040C0C0C81
:1066E0000C0C00078001400040004000000000004A
:1066F000E000E000E00000000000000000000000FA
:1067000000000000E00018030C02CC0564056605DB
:10671000A605B604B604B604B604B602E4010C0439
:106720000C021803F0000000000000000000000050
:10673000000000000000600060005000D0009000E9
:106740009000880088010801F80104030403040292
:10675000020202060F0F000000000000000000000F
:10676000000000000000FE008C030C030C030C036F
:106770000C038C01FC000C030C020C060C060C062E
:106780000C060C03FE0100000000000000000000E9
:10679000000000000000E00318030C060C040404D1
:1067A00006000600060006000600060006040C04AB
:1067B0000C021803F00000000000000000000000C0
:1067C0000000000000007F008C010C030C030C068D
:1067D0000C060C060C060C060C060C060C060C032C
:1067E0000C038C017F00000000000000000000008E
:1067F000000000000000FF03060306040604060074
:1068000086008600FE0086008600860006000604DC
:1068100006040602FF030000000000000000000064
:10682000000000000000FF03060306040604060043
:1068300086008600FE0086008600860006000600B0
:10684000060006001F00000000000000000000001D
:10685000000000000000F00018010C020C0204020D
:106860000600060006000600C60F060306030C031A
:106870000C031803F00000000000000000000000FE
:106880000000000000000F0F0606060606060606BA
:1068900006060606FE07060606060606060606069F
:1068A000060606060F0F00000000000000000000B2
:1068B000000000000000FC03600060006000600059
:1068C00060006000600060006000600060006000C8
:1068D00060006000FC0300000000000000000000F9
:1068E000000000000000F807C000C000C000C000A9
:1068F000C000C000C000C000C000C000C000C00098
:10690000C000C000C000C60066003C0000000000DF
:10691000000000000000CF038601C60046002600EC
:10692000160036002E006E004600C6008600860166
:10693000060106038F0700000000000000000000B1
:106940000000000000001F00060006000600060010
:106950000600060006000600060006000600060403
:1069600006040602FF030000000000000000000013
:106970000000000000000707860386038E038E03D5
:106980004E034E034A035A035A033A0332033203B7
:10699000320312038707000000000000000000001F
:1069A0000000000000008E0F0C021C021C023402CA
:1069B0003402640264024402C40284028403840335
:1069C000040304031F020000000000000000000098
:1069D000000000000000F00098010C030C02060605
:1069E00006060606060606060606060606060C0245
:1069F0000C039801F00000000000000000000000FF
:106A0000000000000000FF0006030606060606065A
:106A1000060606068603FE000600060006000600BF
:106A2000060006001F00000000000000000000003B
:106A3000000000000000F00098010C030C020606A4
:106A400006060606060606060606060676064C0234
:106A5000CC039801F0008007000300000000000054
:106A6000000000000000FF010603060606060606F9
:106A700006060603FE004600C600860086010603E1
:106A8000060306060F0E00000000000000000000D4
:106A9000000000000000F8020C03060206020600D7
:106AA0000E003C00F800E003800300070206020627
:106AB00006060C03F00100000000000000000000CA
:106AC000000000000000FE07620461086108600029
:106AD00060006000600060006000600060006000B6
:106AE00060006000F80100000000000000000000ED
:106AF0000000000000001E070C020C020C020C0239
:106B00000C020C020C020C020C020C020C020C0215
:106B10000C021801F000000000000000000000005E
:106B20000000000000000F070602040104010C0130
:106B30000C018800880098009800500050007000F8
:106B400030002000200000000000000000000000D5
:106B5000000000000000F70E6204420446044604F0
:106B600064026402E402E4029C029C019801980120
:106B7000880188008800000000000000000000007C
:106B80000000000000009E070C01080118019000A1
:106B9000B0006000200060006000D000900088011C
:106BA000080104038E070000000000000000000040
:106BB0000000000000000F0F060404020C02080190
:106BC0001801B800B0007000600060006000600054
:106BD00060006000F80100000000000000000000FC
:106BE000000000000000FC070C0206030201800107
:106BF0008000400040002000200010001800080421
:106C00000C040402FE03000000000000000000006D
:106C1000E0032000200020002000200020002000B1
:106C20002000200020002000200020002000200064
:106C30002000200020002000E003000000000000F1
:106C4000000000000400040008000800100010000C
:106C500010002000200040004000C00080008000A4
:106C60000001000100020002000200040000000018
:106C70007C004000400040004000400040004000D8
:106C80004000400040004000400040004000400004
:106C900040004000400040007C0000000000600018
:106CA000900008010000000000000000000000004B
:106CB00000000000000000000000000000000000D4
:106CC00000000000000000000000000000000000C4
:106CD00000000000000000000000000000000000B4
:106CE00000000000000000000000000000000000A4
:106CF00000000000000000000000FF0F0000000086
:106D0000180060000000000000000000000000000B
:106D10000000000000000000000000000000000073
:106D20000000000000000000000000000000000063
:106D30000000000000000000000000000000000053
:106D4000F0010C030C030003E0031C030E03060315
:106D500006038E0B7C0E0000000000000000000007
:106D60000000000008000E000C000C000C000C00DD
:106D7000CC013C031C060C060C060C060C060C068B
:106D80000C021C03E40100000000000000000000F1
:106D900000000000000000000000000000000000F3
:106DA000F0008C018C018601060006000600060238
:106DB0000C020C01F00000000000000000000000C8
:106DC000000000000002C0030003000300030003F2
:106DD00078038C030C03060306030603060306036D
:106DE00004038C0778010000000000000000000090
:106DF0000000000000000000000000000000000093
:106E0000E001180308020C060C06FC070C000C003D
:106E100018041802E001000000000000000000005B
:106E2000000000000000C0036006300630003000A3
:106E3000FE01300030003000300030003000300003
:106E400030003000FC0100000000000000000000E5
:106E50000000000000000000000000000000000032
:106E6000F007D8068C018C018C019801F8000C0009
:106E7000FC00CC03060306038E03F80000000000AC
:106E80000000000008000E000C000C000C000C00BC
:106E9000EC011C030C030C030C030C030C030C038C
:106EA0000C030C039E07000000000000000000001F
:106EB00000000000000060006000000000004000D2
:106EC0007C006000600060006000600060006000A6
:106ED00060006000FC0300000000000000000000F3
:106EE000000000000000C001C0010000000000011F
:106EF000F00180018001800180018001800180011A
:106F00008001800180018001CC007C000000000035
:106F10000000000008000E000C000C000C000C002B
:106F20008C038C008C004C006C005C008C008C018D
:106F30000C010C039E070000000000000000000090
:106F40000000000040007C00600060006000600005
:106F50006000600060006000600060006000600031
:106F600060006000FC030000000000000000000062
:106F70000000000000000000000000000000000011
:106F80003707EE0666066606660666066606660647
:106F900066066606FF0F000000000000000000000B
:106FA00000000000000000000000000000000000E1
:106FB000EE011C030C030C030C030C030C030C0369
:106FC0000C030C039E0700000000000000000000FE
:106FD00000000000000000000000000000000000B1
:106FE000F00098010C0306060606060606060606CD
:106FF0000C030C03F0000000000000000000000083
:107000000000000000000000000000000000000080
:10701000EE011C030C060C060C060C060C060C06F6
:107020000C031C03EC010C000C003E0000000000EF
:107030000000000000000000000000000000000050
:1070400078028C030C0306030603060306030603FB
:1070500004038C03780300030003C0070000000052
:107060000000000000000000000000000000000020
:107070009F0358063806180018001800180018005A
:1070800018001800FF0000000000000000000000D1
:1070900000000000000000000000000000000000F0
:1070A000F0031C030C020C023800F000C0030403C0
:1070B00004038C03FC01000000000000000000003D
:1070C0000000000000000000200020003000300020
:1070D000FE01300030003000300030003000300061
:1070E00030023002E001000000000000000000005B
:1070F0000000000000000000000000000000080286
:107100008E030C030C030C030C030C030C030C0385
:107110000C039C0778010000000000000000000044
:10712000000000000000000000000000000000005F
:107130001E070C020801080118019000B000B00001
:10714000600060002000000000000000000000005F
:10715000000000000000000000000000000000002F
:10716000F70E6204460464026402EC029C0198017A
:1071700098019801080000000000000000000000D5
:1071800000000000000000000000000000000000FF
:10719000BC0718011001B00060006000E000900022
:1071A000080108039E070000000000000000000026
:1071B00000000000000000000000000000000000CF
:1071C0009E0708010801080190009000B0006000CF
:1071D000600060002000200024001C00000000006F
:1071E000000000000000000000000000000000009F
:1071F000FC018401C400440060002000300018023B
:1072000008020C03FC010000000000000000000068
:1072100000038000800080008000800080008000EB
:10722000800040002000400080008000800080003E
:1072300080008000800080000003000040004000CB
:10724000400040004000400040004000400040003E
:10725000400040004000400040004000400040002E
:10726000400040004000400040004000000000009E
:107270000C00100010001000100010001000100092
:10728000100020004000200010001000100010002E
:1072900010001000100010000C00000000001C0086
:1072A0002204C2048003000000000000000000006F
:1072B00000000000000000000000000000000000CE
:1072C00000000000000000000000000000000000BE
:1072D00000000000000000000000000000000000AE
:1072E000000000000000000000000000000000009E
:1072F000000000000000000000000000000000008E
:10730000000000000000000000000000000000007D
:10731000000000000000C001C001C001C001C001A8
:10732000C001C001800080008000800080008000DB
:10733000800000000000000000008001C003C003C6
:1073400080010000000000000000000000000000BC
:107350000000E01CE01CF01E700E38071803080146
:107360008400000000000000000000000000000099
:10737000000000000000000000000000000000000D
:1073800000000000000000000000000000000000FD
:10739000000000000000000020102010201020102D
:1073A0002010FE7FFE7F100810081008100810083B
:1073B00010081008FE7FFE7F080408040804080473
:1073C00008040000000000000000000000000000B1
:1073D0000000000000010001C007601910311831E1
:1073E0001839183938017001E001C0038007000F17
:1073F000001D003900311C311C310C310C11180DED
:10740000E007000100010001000000000000000092
:1074100000000000000000001C1036186308630C18
:1074200063046304630263026301361D9C37802298
:10743000806340634063206320633063102218360A
:10744000081C000000000000000000000000000018
:107450000000000000000000F00098018C018C0189
:107460008C018C018C00CC007800183E1C0836087A
:10747000320863046304C304C303834306438E26B4
:10748000781C000000000000000000000000000068
:1074900000001C003C003C003000300010000C00DC
:1074A00006000000000000000000000000000000D6
:1074B00000000000000000000000000000000000CC
:1074C00000000000000000000000000000000000BC
:1074D00000000040002000100008000C000400061E
:1074E000000300030003800180018001800180010E
:1074F00080018001800100030003000300060006F4
:10750000000C0008001000200040000000000000F7
:10751000000002000400080010003000200060009D
:10752000C000C000C0008001800180018001800196
:10753000800180018001C000C000C00060006000C8
:1075400030001000080004000200000000000000ED
:1075500000000000000000000000000000018003A7
:10756000800300011C713C79783DC0070001C00711
:10757000783D3C791C71000180038003800100008C
:1075800000000000000000000000000000000000FB
:1075900000000000000000000000000000000001EA
:1075A000000100010001000100010001FC7F000159
:1075B00000010001000100010001000100000000C5
:1075C00000000000000000000000000000000000BB
:1075D00000000000000000000000000000000000AB
:1075E000000000000000000000000000000000009B
:1075F0000000000000000000000000001C003C0033
:107600003C003000300010000C00060000000000BC
:10761000000000000000000000000000000000006A
:10762000000000000000000000000000FE7F0000DD
:10763000000000000000000000000000000000004A
:10764000000000000000000000000000000000003A
:10765000000000000000000000000000000000002A
:10766000000000000000000000000000000000001A
:107670000000000000000000000018003C003C007A
:1076800018000000000000000000000000000000E2
:1076900000000040006000200030001000180008CA
:1076A000000C0004000600020003000180018000BD
:1076B000C0004000600020003000100018000800EA
:1076C0000C000400060002000000000000000000A2
:1076D0000000000000000000C007600C30181830E7
:1076E000183018200C600C600C600C600C600C6092
:1076F0000C600C600C601820183018303018600CCA
:10770000C0070000000000000000000000000000B2
:10771000000000000000000000018001F80180016D
:107720008001800180018001800180018001800151
:107730008001800180018001800180018001C003FF
:10774000F81F000000000000000000000000000022
:107750000000000000000000E007101C08180430C2
:1077600004300C300C300030001800080004000217
:107770000001800040002020102008200430FC1F61
:10778000FC1F0000000000000000000000000000DE
:107790000000000000000000E003180E0C0C0C18A4
:1077A0000C180C180018000C0006C003000E00187E
:1077B0000010003000300C300C300C100C18180C7D
:1077C000E0030000000000000000000000000000D6
:1077D0000000000000000000000C000E000E000F72
:1077E000800E800E400E600E200E100E100E080E41
:1077F000040E040EFE7F000E000E000E000E000EA2
:10780000000EC07F0000000000000000000000002B
:107810000000000000000000F03FF03F10001000EA
:10782000100008000800C807280C181808100030BD
:107830000030003000300C300C3004180418080CF4
:10784000F003000000000000000000000000000045
:107850000000000000000000800FC0102030103039
:107860001800180008000C008C0F6C183C301C60CD
:107870000C600C600C600C601860182030306018D0
:10788000C007000000000000000000000000000031
:107890000000000000000000F83FF83F1C100C083A
:1078A00004080404000400020002000100010001B9
:1078B000800080008000C000C000C000C000C00088
:1078C000C0000000000000000000000000000000F8
:1078D0000000000000000000E007300C18180C3019
:1078E0000C300C301C3038187008E007B007180E48
:1078F0000C1C063806300630063006300C18180C02
:10790000E003000000000000000000000000000094
:107910000000000000000000E00318040C080C1830
:107920000610063006300630063006380C3C183695
:10793000F03100300018001800180C0C0C060C0375
:10794000F001000000000000000000000000000046
:107950000000000000000000000000000000000027
:107960000000000000008001C003C003800100008F
:10797000000000000000000000008001C003C00300
:107980008001000000000000000000000000000076
:1079900000000000000000000000000000000000E7
:1079A000000000000000C000C00000000000000057
:1079B0000000000000000000000000000000C00007
:1079C000C000800080004000400000000000000077
:1079D0000000000000000020001000080004000665
:1079E00000038001C0006000300018000C00180087
:1079F00030006000C00080010003000600040008A1
:107A00000010002000000000000000000000000046
:107A10000000000000000000000000000000000066
:107A2000000000000000FE7F0000000000000000D9
:107A30000000FE7F000000000000000000000000C9
:107A40000000000000000000000000000000000036
:107A5000000000000000040008001000200060008A
:107A6000C000800100030006000C00180030001860
:107A7000000C000600038001C00060002000100020
:107A800008000400000000000000000000000000EA
:107A9000000000000000C0073018083008600C60CB
:107AA0001C601C601C600030001C0006000180008F
:107AB000800080008000000000008001C003C0033F
:107AC0008001000000000000000000000000000035
:107AD0000000000000000000C007601810301820EF
:107AE0000C2F8C4D864CC64CC64C664C6644664486
:107AF000662666266615CC1C0C4008201830301807
:107B0000C0070000000000000000000000000000AE
:107B10000000000000000001C001C001C0014001E0
:107B20006003200320032003300610061006100611
:107B3000F80F080C080C080C0C0C04180418061894
:107B40001F7C00000000000000000000000000009A
:107B50000000000000000000FE07181C1838183054
:107B60001830183018301818180CF8071818183072
:107B700018201860186018601860186018301818FD
:107B8000FE0F0000000000000000000000000000E8
:107B90000000000000000000C027603810301820EE
:107BA0000C400C400400060006000600060006001B
:107BB0000600060006000C400C400C20183030185F
:107BC000C0070000000000000000000000000000EE
:107BD0000000000000000000FE03180E1818183006
:107BE0001830183018601860186018601860186035
:107BF0001860186018601830183018101818180E0F
:107C0000FE03000000000000000000000000000073
:107C10000000000000000000FE3F1830182018602F
:107C20001840180018081808180CF80F180C180835
:107C300018081800180018001840184018201830AC
:107C4000FE3F0000000000000000000000000000F7
:107C50000000000000000000FE7F1870184018C0EF
:107C600018801800181018101818F81F1818181075
:107C70001810180018001800180018001800180034
:107C80007E00000000000000000000000000000076
:107C90000000000000000000C013701C101018103D
:107CA0000C200C200400060006000600060006005A
:107CB00006FC063006300C300C3018301830300816
:107CC000C0070000000000000000000000000000ED
:107CD00000000000000000003F7E0C180C180C187B
:107CE0000C180C180C180C180C180C18FC1F0C187D
:107CF0000C180C180C180C180C180C180C180C1864
:107D00003F7E0000000000000000000000000000B6
:107D10000000000000000000F81F800180018001C9
:107D2000800180018001800180018001800180014B
:107D3000800180018001800180018001800180013B
:107D4000F81F00000000000000000000000000001C
:107D50000000000000000000E07F000600060006B2
:107D600000060006000600060006000600060006E3
:107D700000060006000600060006000600060006D3
:107D8000000600060E060E038E01FC000000000037
:107D900000000000000000007E7C1818180818047D
:107DA00018061802180198019801D801B803380381
:107DB00018071806180E180C181C18181830183048
:107DC0007EFC000000000000000000000000000039
:107DD00000000000000000007E00180018001800DD
:107DE00018001800180018001800180018001800D3
:107DF00018001800180018001840184018201830F3
:107E0000FE3F000000000000000000000000000035
:107E100000000000000000001FF81C381C381C384F
:107E20001C3C343434343434343674326432643286
:107E300064326431C431C431C431C430C43084309C
:107E40009FFC000000000000000000000000000097
:107E500000000000000000001F7C1C103C103410CB
:107E6000341074106410E410C410C411841184130D
:107E7000041304170416041E041C041C041C041818
:107E80001F180000000000000000000000000000BB
:107E90000000000000000000C003300C181808109B
:107EA0000C300C30066006600660066006600660F6
:107EB0000660066006600C200C3008101818300CA4
:107EC000C0030000000000000000000000000000EF
:107ED0000000000000000000FE0F181818301860A5
:107EE000186018601860186018301818F80F18001B
:107EF00018001800180018001800180018001800C2
:107F00007E000000000000000000000000000000F3
:107F10000000000000000000C003300C18180C1016
:107F20000C300C2006600660066006600660066085
:107F3000066006600660E4612C331C321816300EB1
:107F4000C007004C007C003800000000000000006A
:107F50000000000000000000FE07181C1838183050
:107F60001830183018301818180CF8079803180330
:107F7000180718061806180E180C180C181C1818D4
:107F80007E780000000000000000000000000000FB
:107F90000000000000000000E027303818300C20FE
:107FA0000C200C000C0018007800E003800F001E6D
:107FB00000380070006004600460086018303818F1
:107FC000C80F0000000000000000000000000000DA
:107FD0000000000000000000FC3F8C218461824111
:107FE0008241800180018001800180018001800147
:107FF0008001800180018001800180018001800179
:10800000E007000000000000000000000000000089
:1080100000000000000000003F7C0C100C100C1051
:108020000C100C100C100C100C100C100C100C1070
:108030000C100C100C100C100C100C10080838044C
:10804000E00300000000000000000000000000004D
:1080500000000000000000003EF818201820182042
:108060003010301030103010600860086008E00CEC
:10807000C004C004C00480038003800380030001A7
:1080800000010000000000000000000000000000EF
:108090000000000000000000DFF3866186218621D9
:1080A0008C210C218C238C138C138C134C135812A1
:1080B0005816580E380E380E380E300C10041004B6
:1080C000100400000000000000000000000000009C
:1080D00000000000000000007E3E18083808300450
:1080E000300470026002E001C001C0018001800321
:1080F0004003400720062006100C100C0818081832
:108100003E7C0000000000000000000000000000B5
:1081100000000000000000007E7C1C1018101808F1
:108120003008300C700460046002C002C002C0015C
:108130008001800180018001800180018001800137
:10814000E007000000000000000000000000000048
:108150000000000000000000F83F18180818040C88
:10816000040E00060007000380038001C001C00068
:10817000E000600070003000382018201C100C183F
:10818000FE1F0000000000000000000000000000D2
:108190000000C03F40004000400040004000400060
:1081A00040004000400040004000400040004000CF
:1081B00040004000400040004000400040004000BF
:1081C000400040004000C03F0000000000000000F0
:1081D0000000000000000800180018001000300027
:1081E0002000600060004000C0008000800180012D
:1081F000000100030002000600060004000C000855
:1082000000180018001000300020000000000000DE
:108210000000FC0300020002000200020002000253
:10822000000200020002000200020002000200023E
:10823000000200020002000200020002000200022E
:10824000000200020002FC03000000000000000029
:1082500000008007C0062008101000000000000089
:10826000000000000000000000000000000000000E
:1082700000000000000000000000000000000000FE
:1082800000000000000000000000000000000000EE
:1082900000000000000000000000000000000000DE
:1082A00000000000000000000000000000000000CE
:1082B00000000000000000000000000000000000BE
:1082C00000000000000000000000FFFF00000000B0
:1082D00000007800C0000001000000000000000065
:1082E000000000000000000000000000000000008E
:1082F000000000000000000000000000000000007E
:10830000000000000000000000000000000000006D
:10831000000000000000000000000000000000005D
:10832000000000000000F00318060C0C0C0C000C00
:10833000800F700C1C0C0C0C060C060C064C0C4F21
:10834000F8380000000000000000000000000000FD
:1083500000000000000010001E00180018001800A7
:10836000180018001800180FD81838303860186036
:108370001860186018601860186018203830781875
:10838000C80700000000000000000000000000001E
:1083900000000000000000000000000000000000DD
:1083A000000000000000C007700C181818180C1806
:1083B0000C000C000C000C000C20182018103008C9
:1083C000C0070000000000000000000000000000E6
:1083D0000000000000000010001E00180018001827
:1083E000001800180018E01B301C181818180C187A
:1083F0000C180C180C180C180C180818181C307ACB
:10840000E009000000000000000000000000000083
:10841000000000000000000000000000000000005C
:10842000000000000000C007300C181808100C30C5
:108430000C30FC3F0C000C000C00182018107018B9
:10844000C007000000000000000000000000000065
:108450000000000000000000003E80C380C0C0C0DB
:10846000C000C000C000FC1FC000C000C000C000B1
:10847000C000C000C000C000C000C000C000C000FC
:10848000F80F0000000000000000000000000000E5
:1084900000000000000000000000000000000000DC
:1084A000000000000000C077306C10181818181871
:1084B00018181018300CF00718001800F00FF03FD3
:1084C00008700C600C600C603838E00F0000000091
:1084D00000000000000010001E0018001800180026
:1084E000180018001800980FD818383018301830B5
:1084F000183018301830183018301830183018303C
:108500007EFC0000000000000000000000000000F1
:1085100000000000000000008003800380030000D2
:10852000000000000001F80180018001800180014D
:108530008001800180018001800180018001800133
:10854000F81F000000000000000000000000000014
:108550000000000000000000003800380038000073
:10856000000000000010801F0018001800180018FC
:10857000001800180018001800180018001800183B
:10858000001800180018180C1806F003000000006E
:1085900000000000000010001E0018001800180065
:1085A000180018001800183E180C180618031801B7
:1085B0009801D801380318071806180C181C181849
:1085C0007E7C0000000000000000000000000000B1
:1085D0000000000000000001F8018001800180011E
:1085E0008001800180018001800180018001800183
:1085F0008001800180018001800180018001800173
:10860000F81F000000000000000000000000000053
:10861000000000000000000000000000000000005A
:10862000000000000800EE1C9C338C318C318C3132
:108630008C318C318C318C318C318C318C318C3152
:10864000DE7B0000000000000000000000000000D1
:10865000000000000000000000000000000000001A
:108660000000000010001E0FD818383018301830E5
:1086700018301830183018301830183018301830BA
:108680007EFC000000000000000000000000000070
:1086900000000000000000000000000000000000DA
:1086A000000000000000C007701C103018300C6083
:1086B0000C600C600C600C600C60183018303018C6
:1086C000C0070000000000000000000000000000E3
:1086D000000000000000000000000000000000009A
:1086E0000000000010009E0F581838301820186045
:1086F00018601860186018601860183038307818E2
:10870000980718001800180018007E0000000000EC
:108710000000000000000000000000000000000059
:10872000000000000000C023303C183818300C3026
:108730000C300C300C300C300C3008301838303C19
:10874000E033003000300030003000FC000000005A
:108750000000000000000000000000000000000019
:108760000000000060007E3C60666061E000E000A8
:1087700060006000600060006000600060006000F9
:10878000FE070000000000000000000000000000E4
:1087900000000000000000000000000000000000D9
:1087A000000000000000E0273038183018201800C2
:1087B0007000E003800F001C043004300C301C18E3
:1087C000EC0F0000000000000000000000000000AE
:1087D0000000000000000000000000008000800099
:1087E0008000C000E000FC1FC000C000C000C0004E
:1087F000C000C000C000C000C000C020C020801168
:10880000000F000000000000000000000000000059
:108810000000000000000000000000000000000058
:108820000000000010201E3C18301830183018309E
:10883000183018301830183018301830183830F414
:10884000E013000000000000000000000000000035
:108850000000000000000000000000000000000018
:108860000000000000007E3C18181808380830048A
:108870003004700260026002E001C001C001C0006B
:108880008000000000000000000000000000000068
:1088900000000000000000000000000000000000D8
:1088A000000000000000DFF78E630C238C238C2374
:1088B0009813981358165816700E700E700E2004E8
:1088C0002004000000000000000000000000000084
:1088D0000000000000000000000000000000000098
:1088E000000000000000FC3E70087004E004C002BC
:1088F000C0018003800340076006200C100C18188C
:108900003E7E0000000000000000000000000000AB
:108910000000000000000000000000000000000057
:108920000000000000007E7C18181808300830088D
:10893000300460046004C002C002C00280018001F3
:1089400080018000800080004C003C00000000009E
:108950000000000000000000000000000000000017
:10896000000000000000FC1F0C0C040E04060003B5
:1089700080038001C000E0007020302038301C18D7
:10898000FC1F0000000000000000000000000000CC
:10899000000000300008000400040004000400048B
:1089A000000400040004000400040002800100022E
:1089B0000004000400040004000400040004000497
:1089C0000004000400040008003000000001000161
:1089D000000100010001000100010001000100018F
:1089E000000100010001000100010001000100017F
:1089F000000100010001000100010001000100016F
:108A00000001000100010001000100010000000060
:108A100000000C001000200020002000200020009A
:108A200020002000200020002000400080014000A5
:108A30002000200020002000200020002000200036
:108A400020002000200010000C0000000000380072
:108A5000C400864002610022001C000000000000EB
:108A60000000000000000000000000000000000006
:108A700000000000000000000000000000000000F6
:108A8000000000000000000000000000D6D0200020
:108A900020002000FE03220222022202FE03220204
:108AA000200020002000BEB0FC010401FC010401F4
:108AB000FC012000FF070401FC0120002401320218
:108AC000D4B0FE070204FA0402040204FE055204B4
:108AD00052044A0586050204FE07B5E7100010009F
:108AE000FF0111011101FF0111011101FF01110429
:108AF0001004E007D7D30000FC01800040002000F4
:108B00002000FF0720002000200020003800D6D0E1
:108B10008000800080008000FC1F8410841084107E
:108B200084108410FC1F841080008000800080006E
:108B3000BEB0F80F0808F80F0808F80F8000FF7F94
:108B40000000F80F08080808F80F80008410A22021
:108B50004000D4B00000FE3F0220F2270220022095
:108B6000FA2F222122212221122912290A2E022043
:108B7000FE3F0220B5E7800080008000FC1F8410CB
:108B800084108410FC1F841084108410FC1F8450F7
:108B900080408040007FD7D30000FE1F0008000403
:108BA000000280018000FF7F800080008000800044
:108BB00080008000A0004000D6D00000000000002F
:108BC000001800000800000800000800080818F855
:108BD000FF1F180818180818180818180818180877
:108BE00018180818F8FF1F080808000800000800F7
:108BF000000800000800001800001800001800001D
:108C00000000BEB0000000000000400006C0FF07EA
:108C1000400006C0FF07400006C0FF0740080200F2
:108C20003000FEFF3F000000C0FF07C00002C00090
:108C300002C00002C0FF0380100080110160100E0E
:108C40003010180C1E30001C00000000D4B00000D2
:108C500000000000080030F8FF1F08001008C010D6
:108C6000083F10080010080010080013C8FF100883
:108C700022100822100822100822100821120821B0
:108C80001488601648C013280010080010F8FF1F51
:108C9000080010000000B5E7000000000000001808
:108CA00000000800000800000800F0FF0F10080492
:108CB000100804100804100804F0FF07100804103E
:108CC0000804100804100804F0FF0710080000084A
:108CD0001000081000082000183000F01F000000ED
:108CE000D7D3000000000000000004F0FF0F0000D8
:108CF0000600000100C00000280000180000180055
:108D0000001830FEFF7F0018000018000018000057
:108D100018000018000018000018000018000018C3
:108D200000001F00000C00000000D6D00000000072
:108D300000000000008000000080010000800100B1
:108D40000080010000800100008001001080010C03
:108D5000F0FFFF0F308001043080010430800104F7
:108D6000308001043080010430800104308001042F
:108D700030800104F0FFFF073080010430800104DF
:108D800000800100008001000080010000800100DF
:108D900000800100008001000080010000800100CF
:108DA000008001000080000000000000BEB0000054
:108DB000000000000000000000000001800100FF32
:108DC000FF01000380010003800100FFFF01000399
:108DD00080010003800100FFFF010081810000008D
:108DE00003000000031CFCFFFF3F000040000003E5
:108DF000C00100FFFF010003C0000003C00000032A
:108E0000C00000FFFF000001410000040100000E4F
:108E1000710000078101800101076000010E1898B0
:108E2000011C04E0011800C0000000000000D4B0E4
:108E3000000000000000000000000008F0FFFF1F1D
:108E40003000000C3000000C3000100C30FE3F0CE5
:108E50003004000C3000000C3000000C3000000C1E
:108E60003000C00CF0FFFF0D3030060E3030060C25
:108E70003010060C3010060C3010060C3018860C22
:108E80003018860C3008060D300C860D3006EE0FBB
:108E90003002FC0D3001000CF000000C3000000C22
:108EA000F0FFFF0F3000000C100000040000000075
:108EB000B5E7000000000000000000C0000000C096
:108EC000010000C0000000C0000000C0000000C0A1
:108ED0000000E0FFFF0360C0000360C0000360C04B
:108EE000000360C0000360C0000360C00003E0FF37
:108EF000FF0360C0000360C0000360C0000360C0E7
:108F0000000360C00003E0FFFF0360C0000160C019
:108F1000000000C0000800C0001000C0001000C029
:108F2000001800C001380080FF1F00000000000092
:108F30000000D7D300000000000000000000000087
:108F400000000003C0FFFF07000080070000C00012
:108F5000000060000000180000000C00008003000A
:108F60000080030000800100008001080080011CD7
:108F7000FCFFFF3F00800100008001000080010035
:108F800000800100008001000080010000800100DD
:108F900000800100008001000080010000800100CD
:108FA0000080010000FC010000E000000040000023
:108FB00000000000D48F00080000002084000000A2
:108FC000D001000858900008840000202478000098
:108FD000EC0100080000000010000000010000008B
:108FE00000093D000000000000000000000000003B
:108FF0000000000000000000000000000000000071
:109000000000000000000000000000000000000060
:1090100010270000102700000000000000000000E2
:109020000000000000000000000000000000000040
:109030000000000000000000000000000000000030
:109040000000000000000000000000000000000020
:08905000000000000000000018
:040000050800019559
:00000001FF
